:100000000C94D6050C94F5050C94F5050C94F505A7
:100010000C94F5050C94F5050C94F5050C94F50578
:100020000C94F5050C94F5050C94200A0C94F50538
:100030000C94F5050C94F5050C94F5050C94F50558
:100040000C94F5050C9432070C944B2E0C941B2E3B
:100050000C94F5050C94F5050C94F5050C94F50538
:100060000C94F5050C94F5050C94F5050C94F50528
:100070000C94F5050C94F5050C94F5050C94F50518
:100080000C94F5050C94F5050C94F5052A29B02B74
:100090003529B02B51295129A929ED292C2A7C2A4F
:1000A000BE29B02BB02B142B252B4B2B602BB02B48
:1000B000B02BB02BB02BB02BB02BB02BB02BB02B68
:1000C000B02BB02BB02B9C2B9E2BA32B712B312E46
:1000D000342E3700696E636F6D70617469626C6590
:1000E000204857002020253032580020504300205F
:1000F0004C430045617379436F6E74726F6C0001FD
:1001000002031718040506151107080916120A003C
:100110000B0C13100F0E0D14040E1F0E0E0E0E00FE
:100120000E0E0E0E1F0E0400080C1E1F1E0C0800E3
:1001300002060F1F0F0602000E11111F1B1B1F00CE
:100140001F0A0A0A0A0A1F001C10181016050505C6
:100150000C17141714170C00040A110A0A0E0000D9
:100160001C101812160202071C10181611020407A0
:100170001C101816110201061C1018151507010194
:1001800000000017151515171212121212000000A8
:100190000000001711171417171113111700000092
:1001A0000000001515171111171417111700000082
:1001B00007050505050505070707070707070707DB
:1001C000030509121418100003070F1E1C18100055
:1001D000000609121412090600060917170906007D
:1001E000040E1F04041F0E04010101050D1F0C0461
:1001F00011040A11111F1100110E111111110E001D
:100200000A00111111110E000E1111161111161004
:10021000206D332020200000204D4D49202000007B
:10022000204D4D02202000002044434320200000A8
:100230002053544F5020000053484F525421000087
:100240002048414C54200000202020202020000085
:100250002050524F47200000524553455420000083
:10026000202054504D200000202020200025336401
:1002700000252D31312E31317300252D3564004696
:10028000253032643D2563002020010220202020FB
:10029000202020002533640025336400252D35649B
:1002A000002D2D2D2D2020004144523A20256C6434
:1002B0002020202020202020202000232D007E0E22
:1002C0000E0E0E1B1B1C0E1B1B7E0E0E0E0E25355E
:1002D0007500202D2D2D2D004142434445464748B1
:1002E000494A4B4C4D4E4F50515253545556575806
:1002F000595A303132333435363738392E2C3A2D7D
:100300002B232F3D3C7C3E20004D4D2049202031A9
:100310003420004D4D20492020323761004D4D20C2
:10032000492020323762004D4D20022020313420F8
:10033000004D4D20022020323761004D4D2002201B
:1003400020323762004443432020203134200044CF
:1003500043432020203238200044434320203132C0
:100360003820006D3320202031323820003A200020
:10037000253575005365724E722E2025386C750038
:10038000312E342E3700536F6674772E2056002599
:1003900033640025346400202D2D2D0020202020E2
:1003A00020202000204F4B202020200025336400F7
:1003B0002D2D2D002534643A20004C6F6B204D65A7
:1003C0006EFC000000000000000044434320486130
:1003D000757074676C656973000044434320526113
:1003E000696C436F6D204356000045696E737465F8
:1003F0006C6C756E67656E0000004C43442042656E
:100400006C6575636874756E67004C6F6B436F6ED7
:1004100074726F6C00000000000045786974000081
:100420000000000000000000000041757377E468E0
:100430006C656E20000000000000446174656E660B
:100440006F726D617400000000004E616D652020C8
:100450002020202000000000000045696E747261B9
:100460006720202000000000000031323846532071
:100470004D6F64650000000000005265676C657296
:100480006D6F64757300000000004D656E75204C43
:100490006F636F0000000000000050726F677261B0
:1004A0006D6D6174696F6E000000444343205261BA
:1004B000696C436F6D20435600005265676C61673D
:1004C000657300000000000000004C756D696E6FE0
:1004D000736974650000000000004C6F6B436F6E21
:1004E00074726F6C000000000000457869740000B1
:1004F0000000000000000000000053656C6563749C
:10050000696F6E20000000000000466F726D61741C
:1005100020646F6E6E65657300004E6F6D20202045
:1005200020202020000000000000536169736965ED
:1005300020202020000000000000313238465320E7
:100540004D6F64650000000000004A6F67646961D8
:100550006C204D6F6465000000004C6F636D656E2C
:100560007500000000000000000044434320686F55
:100570006F666473706F6F72000044434320526172
:10058000696C436F6D2043560000496E7374656C4F
:100590006C696E67656E000000004C434420766510
:1005A000726C69636874696E67004C6F6B436F6E41
:1005B00074726F6C000000000000457869740000E0
:1005C000000000000000000000004B69657A656EC5
:1005D0002000000000000000000044617461666FAC
:1005E000726D61740000000000004E61616D20209A
:1005F00020202020000000000000496E766F657208
:100600002020202000000000000031323846532016
:100610004D6F64650000000000004A6F6764696107
:100620006C204D6F6465000000004C6F636F6D6F50
:1006300074697665206D656E7500444343204D6195
:10064000696E20547261636B000044434320526121
:10065000696C436F6D204356000053657474696E76
:10066000677300000000000000004C4344206261FA
:10067000636B6C696768740000004C6F6B436F6E4E
:1006800074726F6C0000000000004578697400000F
:100690000000000000000000000053656C656374FA
:1006A000200000000000000000004461746120662A
:1006B0006F726D617400000000004E616D65202056
:1006C00020202020000000000000456E7472792078
:1006D0002020202000000000000031323846532046
:1006E0004D6F64650000000000004A6F6764696137
:1006F0006C204D6F646500000000696E6B6F6D705B
:1007000061742E20466F726D617400466F726D6168
:100710007420696E636F6D7061742E00496E636F33
:100720006D702E20466F726D6174202000696E63BB
:100730006F6D7061742E20466F726D6174005B7511
:100740006E6B6E6F776E206572726F725D002E2E0B
:100750002E2077617274656E202E2E2E20200023AD
:100760003D4CF6736368656E0000000000000000F9
:10077000286B65696E2045696E7472616729000097
:1007800000202E2E2E206CF673636865202E2E2EF0
:100790002000204665686C657200000000000000C3
:1007A000000000206E75722066FC722044434321D5
:1007B00020202000206572737420474F206472FC53
:1007C000636B656E002A3D4162627275636800006A
:1007D0000000000000002050726F6772616D6D694B
:1007E0006572756E6700002D2D204B75727A7363EC
:1007F000686C75DF202D2D00204E617469762028ED
:10080000313A31292020202000204C696E65617228
:100810002028323A3129202020002050726F677240
:1008200065737369762031202020002050726F6735
:1008300072657373697620322020200020414320A6
:100840004D6F647573202020202020200020444319
:10085000204D6F64757320202020202020005061DF
:100860007469656E74657A00000000000000002362
:100870003D7375707072696D657200000000000054
:1008800076696465000000000000000000000000C0
:10089000005375707072657373696F6E00000000AD
:1008A00000002045727265757200000000000000B3
:1008B0000000002044434320756E697175656D65C5
:1008C0006E74200020707265737320474F20666934
:1008D00072737400002A3D4162616E646F6E0000A5
:1008E0000000000000002050726F6772616D6D6142
:1008F00074696F6E0000002D436F7572742D63690B
:1009000072637569742D2000206E617469766520AC
:1009100028313A312920202000206C696E656172EF
:100920002028323A3129202020002070726F67720F
:1009300065737369766520312020002070726F67BF
:100940007265737369766520322020002041432050
:100950004D6F64652020202020202020002044436B
:10096000204D6F64652020202020202020002E2E86
:100970002E207761636874656E202E2E2E20002352
:100980003D77697373656E00000000000000000091
:10099000286765656E20696E766F657229000000B4
:1009A00000202E2E2E2077697373656E202E2E2E3A
:1009B000000020666F757400000000000000000059
:1009C00000000020416C6C65656E2044434321208B
:1009D0002020200020707265737320474F206669C5
:1009E00072737400002A3D41666272656B656E0029
:1009F0000000000000002050726F6772616D6D652D
:100A000072656E000000002D2D4B6F7274736C7553
:100A10006974696E672D2D00206E6174697665209A
:100A200028313A312920202000206C696E656172DE
:100A30002028323A3129202020002070726F6772FE
:100A400065737369766520312020002070726F67AE
:100A5000726573736976652032202000204143203F
:100A60004D6F64652020202020202020002044435A
:100A7000204D6F64652020202020202020002E2E75
:100A80002E2077616974696E67202E2E2E20002338
:100A90003D64656C657465000000000000000000A6
:100AA000286E6F20656E74727929000000000000C6
:100AB000002E2E2E2064656C6574696E67202E2EC4
:100AC0002E00206661756C740000000000000000BC
:100AD00000000020444343206F6E6C7921202020C9
:100AE0002020200020707265737320474F206669B4
:100AF00072737400002A3D43616E63656C000000F0
:100B00000000000000002070726F6772616D696EF6
:100B1000670000000000002D73686F727420636925
:100B200072637569742D2000206E6174697665208A
:100B300028313A312920202000206C696E656172CD
:100B40002028323A3129202020002070726F6772ED
:100B500065737369766520312020002070726F679D
:100B6000726573736976652032202000204143202E
:100B70004D6F646520202020202020200020444349
:100B8000204D6F64652020202020202020005B6EF7
:100B90006F206D6573736167655D004003A001CFD1
:100BA00000670044003300190010000011241FBE2C
:100BB000CFEFD0E1DEBFCDBF11E0A0E0B1E0E4E6D1
:100BC000FAE600E00BBF02C007900D92A634B10711
:100BD000D9F713E0A6E4B1E001C01D92AC3CB10727
:100BE000E1F70E9415060C9430350C9400008091BA
:100BF0004601089581E080934701089580E00E94B6
:100C00004A0EBC018FEF6F3F780719F080E00E9419
:100C1000FD2F0E94BE270E94B010809147018823BB
:100C200011F40E94FD0CA8950895CF93DF930E94C4
:100C30008E260E94F10683E068E04EE422E00E94E6
:100C4000D82D0E94BF0878940E94D50A0E94612581
:100C5000DC0114968C910E94F80C82E063EF70E046
:100C60000E942C0F0E947925823021F00E94792564
:100C7000813021F482E06FEE70E007C00E94792598
:100C80008038D9F482E06BEE70E00E942C0F81E096
:100C900060E00E947B0D82E066E50E94590E82E0D2
:100CA0006EEC70E00E942C0F0E946125EC0181E047
:100CB0000E94AB0B882349F125C00E94792500D002
:100CC00000D00F92EDB7FEB7319692E0ADB7BEB748
:100CD00011969C9324EE30E0328321838383148227
:100CE0000E94D20E0F900F900F900F900F9081E006
:100CF00060E00E947B0D82E064ED70E00E942C0FAA
:100D0000A895FECF81E00E94752682E00E94AB0B81
:100D1000882319F080E00E94752683E00E94AB0BC7
:100D2000882319F082E00E94752684E00E94AB0BB4
:100D3000882329F083E00E94752601C0A8950E94AF
:100D40000B288823D9F389859A85009749F060E0BC
:100D500070E040E050E00E94412DBC01009711F48A
:100D60006A817B818FEF0E94212681E011C00E9461
:100D7000A0150E94CF0BBFEF8F3F9B07C1F70E94CA
:100D8000FE05809147018823A1F31092470180E07E
:100D90000E948411EECF90914601981701F1963090
:100DA000F1F0953011F48630D1F48093460185300E
:100DB00029F480E060E245E00E94482780914601E6
:100DC000863029F480E060E246E00E944827809166
:100DD00046010E94C02F81E080934701089580E082
:100DE00008958FE78ABB1BBA80E187BB18BA80EFF2
:100DF00084BB8FEF85BB8BEB81BB8CEC82BB82E02D
:100E000082B987EF83B987E78093610081EF809390
:100E100062008FE18093640089E1809365000E9405
:100E20008D09A89588E181BD8EE081BD0895DC0122
:100E300090914B0189E0989FF0011124ED5CFC4FEB
:100E400090E08D9181939F5F9930D9F780914B010C
:100E50008F5F80934B0180914B01843010F0109292
:100E60004B0108951F920F920FB60F920BB60F927F
:100E700011241F932F933F934F935F936F937F930F
:100E80008F939F93AF93BF93EF93FF938091000154
:100E9000909101012FEF8F3F920761F0BB9A8FB9BC
:100EA000769B0BC0BB9810924A0110925001109291
:100EB0004F0103C0BB988FEF8FB91FB117FF8AC0D6
:100EC0008091510190915201892BE1F080914D0167
:100ED0008F5F80934D0180914D01803210F0109210
:100EE0004D0190914D0180914E01981759F48091D8
:100EF0004E018F5F80934E0180914E01803210F041
:100F000010924E0180914F01909150018353934074
:100F100061F058F080914C018F5F80934C0180917B
:100F20004C01843010F010924C011092520110923A
:100F300051011092500110924F01809143011817F6
:100F400021F481E080934A0177C010924A01412F39
:100F500050E04F775070682F70E04617570729F020
:100F60001F3F19F08F3F09F067C080914D0129E0C4
:100F7000829FC00111248D5E9D4F909352018093FA
:100F800051014617570709F057C090914B018091C6
:100F90004C01981721F48AE092E00E941707809193
:100FA0004C0129E0829FC00111248D5C9C4F9093DD
:100FB000500180934F0180914C018F5F80934C01D1
:100FC00080914C01843010F010924C0189E08093A4
:100FD000480132C020914A01213029F0213060F1CE
:100FE000263050F515C082E080934A01103419F480
:100FF0001092490121C0113419F4209349011CC0F9
:10100000123419F0133491F483E08093490114C031
:10101000E22FF0E08091490190E002968E179F0741
:1010200044F0EF5AFE4F8081181719F010924A01D0
:1010300003C02F5F20934A0180914A01882329F041
:10104000109300011092010121C0E0914F01F09135
:1010500050013097A9F08191809300011092010115
:10106000F0935001E0934F018091480181508093AB
:101070004801882359F41092500110924F0106C084
:101080008FEF9FEF9093010180930001E091510158
:10109000F0915201309749F083E0E333F80728F4E8
:1010A0001193F0935201E0935101FF91EF91BF91A1
:1010B000AF919F918F917F916F915F914F913F91F0
:1010C0002F911F910F900BBE0F900FBE0F901F908E
:1010D00018951F93AC011FB7F89420914B01809194
:1010E0004C0130E090E001972817390741F08091DA
:1010F0004B01833039F480914C01882319F41FBFD0
:1011000080E005C0CA010E9417071FBF81E01F9140
:101110000895DC01EAE0F2E08D91819382E0E33111
:10112000F807D1F708959C01009739F14FB7F8946B
:1011300090914D0180914E01981721F44FBF20E00E
:1011400030E01BC090914E0189E0989FF00111247E
:10115000ED5EFD4FD90190E081918D939F5F9930B5
:10116000D9F780914E018F5F80934E0180914E019F
:10117000803210F010924E014FBFC90108950E94B5
:101180006B25262F2F772093560147E0969587955C
:10119000779567954A95D1F7262F2F77209355019C
:1011A00037E096958795779567953A95D1F7262FED
:1011B0002F772093540127E096958795779567952B
:1011C0002A95D1F76F776093530187B3807F87BBF0
:1011D00088B3807F88BB84EE8DB90895882351F051
:1011E000809165008460809365000000000000002D
:1011F00000000895809165008B7F809365000895BD
:101200000F931F93DF93CF930F92CDB7DEB7182FB5
:101210008AB3807F8ABB80E00E94EE0880916500DF
:10122000826080936500112321F0809165008160C8
:1012300003C0809165008E7F8093650000000000F0
:1012400081E00E94EE0809B380E00E94EE0810E001
:1012500084E0000F111F8A95E1F7000000000000F4
:10126000000081E00E94EE0899B39F70902B80E00F
:1012700099830E94EE089981892F0F90CF91DF9179
:101280001F910F91089580E00E940009982F80918E
:101290005A01882331F497FD04C0892F8F778093FA
:1012A0005B01892F881F8827881F08959B01AC0147
:1012B0008091590390915A03A0915B03B0915C0314
:1012C00082179307A407B50798F08091590390916E
:1012D0005A03A0915B03B0915C0360E0821B930B07
:1012E000A40BB50B80509041A040B040A0F412C0B8
:1012F0008091590390915A03A0915B03B0915C03D4
:1013000060E0281B390B4A0B5B0B2050304F4F4FCE
:101310005F4F08F061E0862F089510927D0080B73E
:10132000877F80BF17BE11BE89E683BF82E085BD7F
:1013300087B7806487BF0895EF92FF920F931F9342
:101340002091590330915A0340915B0350915C0303
:101350007C0100E010E0E20EF31E041F151F01C027
:10136000A895C801B7010E9456098823C9F31F91A7
:101370000F91FF90EF900895FF920F931F93082F06
:10138000162FF42E809165008D7F8093650080E09C
:101390000E94EE088AB38F608ABB8BB3902F929520
:1013A0009F70807F982B9BBB112321F0809165005B
:1013B000816003C0809165008E7F8093650081E02D
:1013C0000E94EE0880E00E94EE08FF2029F088E0ED
:1013D00090E00E949C090FC08BB30F70807F802B20
:1013E0008BBB000000000000000081E00E94EE08BE
:1013F00080E00E94EE081F910F91FF900895EF92F8
:10140000FF920F931F932091590330915A034091FB
:101410005B0350915C037C0100E010E0E20EF31EE0
:10142000041F151F02C00E94FE05C801B7010E94DB
:1014300056098823C1F31F910F91FF90EF900895F3
:101440001F920F920FB60F920BB60F9211241F939B
:101450002F933F934F935F936F937F938F939F93BC
:10146000AF93BF93EF93FF9380915701882309F0C7
:1014700088C081E0809357017894809159018F5FF3
:10148000809359018091590190E083709070813070
:101490009105E1F08330910559F1892B09F06FC076
:1014A0008091590390915A03A0915B03B0915C0322
:1014B0000196A11DB11D8093590390935A03A093E7
:1014C0005B03B0935C030E94B70B59C08091590332
:1014D00090915A03A0915B03B0915C03817090706E
:1014E000892B19F00E94E90B4AC00E946F0B47C07C
:1014F00080915801882319F00E9443093EC09091C1
:101500005D0380915E039817B9F180915E03E82F27
:10151000F0E0E35AFC4F9281182F1F5F103108F062
:1015200010E0903801F580915D03811729F1E12FDA
:10153000F0E0E35AFC4F92819F3F19F490915B01D8
:10154000906897FF02C010925A01892F807C8034E6
:1015500019F481E080935A011F5F103108F010E008
:10156000892F60E002C0892F61E040E00E94BC0941
:1015700010935E0381E001C080E0809358011092D7
:101580005701FF91EF91BF91AF919F918F917F9103
:101590006F915F914F913F912F911F910F900BBED3
:1015A0000F900FBE0F901F901895CF93DF9388E296
:1015B00090E00E949C0980E360E041E00E94BC0949
:1015C00080E360E041E00E94BC0980E360E041E02C
:1015D0000E94BC0980E260E041E00E94BC0988E210
:1015E0000E94650D80E40E94650D8AE00E94380D1E
:1015F00089E20E94650D8CE10E94650D82E50E94E2
:10160000650D89E60E94650D84E70E94650D80E402
:101610000E94650D85E10E94380D88E20E94650DEB
:1016200080E40E94650D0E94550FEC0101C0A89551
:1016300090915D0380915E039817C9F70E9443095A
:101640008823A9F781E00E9400098A3019F481E01B
:1016500088AB01C018AA88E00E94650D81E00E9455
:10166000650D86E00E94650D8CE00E94650D80E0AE
:1016700060E00E947B0D80E068E171E00E94280E2E
:1016800081E068E371E00E94280E82E060E471E08E
:101690000E94280E83E060E571E00E94280EDF9131
:1016A000CF91089590915E01E92FF0E0E25AFE4F4C
:1016B00082839F5F90935E01983010F010925E01DC
:1016C00090915F0180915E01981741F4892F8F5F9F
:1016D00080935F01883010F010925F01089531B15E
:1016E00020915D01220F36FD2160822F8370815091
:1016F000823028F424FF02C02E6001C0217F209395
:101700005D0190915C01990F37FD9160892F837085
:101710008150823028F494FF02C09E6001C0917F06
:1017200090935C01207C892F807C203831F48823C1
:1017300041F0803C79F48AE105C0203459F4803CC2
:1017400021F489E10E94520B0895882319F48AE15B
:101750000E94520B0895893110F080E00895E82F1F
:10176000F0E0E859FE4F8081811181E008953091C9
:101770009A01343029F485B3806F85BB979808951A
:10178000979A25B380E190E002C0880F991F3A959F
:10179000E2F78095807F2F70822B85BB0895909112
:1017A0005F0180915E01891719F42FEF3FEF0FC0A1
:1017B000E92FF0E0E25AFE4F8281282F30E0892F96
:1017C0008F5F80935F01883010F010925F01C90134
:1017D00008958F929F92AF92BF92CF92DF92EF9235
:1017E000FF920F931F93CF93DF930E94F705982FDB
:1017F00080919B01981729F090939B0182E20E94AF
:10180000520B83B3E1B0EE0CEE0C90E1E9228F7045
:10181000E82ACC24DD2495E0892E81E0A82EB12C85
:1018200099249394E0919A01E89DF0011124EC0D24
:10183000FD1DE150FF4FF49088E18F1508F481C041
:101840000E2D0A250170CF2DD0E0FE01EF57FE4F7F
:101850001081110F0E947925803819F4002371F04E
:1018600009C001111160812F90E081719070813168
:10187000910511F41F6103C0892B09F4107E812F9B
:1018800090E0807690708034910519F41F7182E0A9
:101890000CC08032910519F4106E81E006C08036CC
:1018A000910511F080E001C083E0FE01EF57FE4F8B
:1018B0001083823099F0833059F1813009F041C0B2
:1018C00096E1F91621F480917D01882319F48F2D7A
:1018D0000E94520BC859DE4F988233C0C859DE4F60
:1018E00018828F2D80680E94520B0E94F705853068
:1018F00041F585E1F81619F480917E0105C096E165
:10190000F916F9F480917D018823D9F486E017C097
:10191000FE01E859FE4F80818F5F8083882309F4A0
:1019200090828BEEF80E91E09F1558F080917D012A
:10193000893738F080917E01893718F085E00E9460
:10194000CB060894C11CD11C85E0C816D10411F047
:10195000E69468CF80919A018F5F80939A018530D9
:1019600010F010929A01DF91CF911F910F91FF908B
:10197000EF90DF90CF90BF90AF909F908F900895A1
:1019800090938A0380938903892B89F1709388034C
:10199000609387038091590390915A03A0915B0350
:1019A000B0915C039B0140E050E0280F391F4A1FB3
:1019B0005B1F2093830330938403409385035093EC
:1019C0008603809182038E7F8093820321153105E7
:1019D0004105510561F481E090E0A0E0B0E0809322
:1019E000830390938403A0938503B09386030895A3
:1019F000813308F080E381BF08958091890390913D
:101A00008A03892BA1F160918303709184038091F3
:101A10008503909186030E945609882341F18091A5
:101A20008203E0918903F0918A0381700995809186
:101A3000820391E08927809382032091590330919A
:101A40005A0340915B0350915C038091870390910E
:101A50008803A0E0B0E0820F931FA41FB51F8093FE
:101A6000830390938403A0938503B0938603089522
:101A70001F93182F03C00E94BE27A89520915D03D5
:101A800080915E0330E090E001972817390799F3C1
:101A900080915D038F3021F480915E03882359F398
:101AA000F894E0915D03F0E0E35AFC4F12838091DB
:101AB0005D038F5F80935D0380915D03803110F043
:101AC00010925D0378941F9108951F93182F80E85A
:101AD0000E94380D812F0E94380D1F910895109299
:101AE0008A031092890381E00E94650D08958CE0BD
:101AF0000E94650D08958295880F880F807C860F5F
:101B000080680E94650D0895BF92CF92DF92EF9298
:101B1000FF920F931F93CF93DF93C82EB62E7A01B7
:101B200010928A031092890381E08C15B8F1EFE0DE
:101B3000E617A0F14115510589F1FA010190002045
:101B4000E9F73197DE2ED41AF0E1FD1510F480E1AB
:101B5000D82E8C2D6B2D0E947B0D0FE613E0CD2D22
:101B6000D0E0C00FD11F0BC0F7018081F801819335
:101B70008F01F70161917F0182E00E94590E0C17DD
:101B80001D0791F7C0927F03B0928003D09281032A
:101B900081E09EE064EF71E00E94C00CDF91CF9184
:101BA0001F910F91FF90EF90DF90CF90BF9008951D
:101BB000DF93CF93CDB7DEB7A0970FB6F894DEBF13
:101BC0000FBECDBFDE0111969E01205E3F4F04C0C7
:101BD0009D93A217B30731F0FA014F5F5F4F9491C5
:101BE0009923B1F71C92AE014F5F5F4F0E94840DA5
:101BF000A0960FB6F894DEBF0FBECDBFCF91DF9198
:101C000008950F931F93CF93DF93082F80917F0345
:101C1000609180030E947B0D10E0CFE6D3E009C005
:101C2000002311F460E201C0699182E00E94590E24
:101C30001F5F80918103181798F3DF91CF911F9157
:101C40000F9108950E947B0D8EE00E94650D08950E
:101C50000F931F93CF93DF938B018830B0F4880FDD
:101C6000880F880F80640E94650DC0E0D0E0F80105
:101C7000EC0FFD1FE4918E2F0E94380D2196C83085
:101C8000D105A9F78FEF0E94650DDF91CF911F91CC
:101C90000F910895882341F0823019F02FEF3FEF24
:101CA00006C00E94CF0B02C00E944B2F9C01C901AD
:101CB00008951F93162F882309F45EC0823009F01F
:101CC0005EC067FF55C00E94550FFC0180A98823A4
:101CD000E1F0143E11F414E84BC0163F11F414E97E
:101CE00047C01C3F11F411E843C0143C11F41EE836
:101CF0003FC0163D11F419E93BC01C3D11F41AE92F
:101D000037C0113F69F51BE933C0143E11F411EEE1
:101D10002FC0163F11F41FEE2BC01C3F11F415EF1E
:101D200027C0113F11F41EEE23C0143C39F484E0A7
:101D300060EF71E00E94280E14E01AC0163D39F4DD
:101D400085E068EF71E00E94280E15E011C01C3D8F
:101D500039F486E060E072E00E94280E16E008C0C8
:101D60001F3D31F487E068E072E00E94280E17E022
:101D7000812F0E94380D03C0862F0E941B2F1F91B8
:101D800008951F93CF93DF93182FEB0104C0219682
:101D9000812F0E94590E68816623C9F7DF91CF9188
:101DA0001F9108950F931F93DF93CF93CDB7DEB7A5
:101DB000C055D0400FB6F894DEBF0FBECDBF9E0118
:101DC000265A3F4F8E010F5F1F4FC8016A966EADB6
:101DD0007FAD6A97A9010E943C3268968FAD6897E3
:101DE000B8010E94C10EC05BDF4F0FB6F894DEBF92
:101DF0000FBECDBFCF91DF911F910F9108950F932B
:101E00001F93DF93CF93CDB7DEB7C055D0400FB649
:101E1000F894DEBF0FBECDBF9E01265A3F4F8E0104
:101E20000F5F1F4FC8016A966EAD7FAD6A97A9011B
:101E30000E94133268968FAD6897B8010E94C10E58
:101E4000C05BDF4F0FB6F894DEBF0FBECDBFCF91A2
:101E5000DF911F910F9108951F93CF93DF93182F58
:101E6000EB0104C0812F0E94590E2196FE0164915E
:101E70006623C1F7DF91CF911F910895E82FF0E01D
:101E8000EF70F070E254FD4FE4918E2F90E00895D2
:101E900090E083709070009731F0039711F48CE11B
:101EA000089584E008958FE008958CE991E0089505
:101EB0008091B80182FF05C080919E0190919F01A1
:101EC000089580919C0190919D0108959091B80191
:101ED00091FD19C092FF05C080918B03823099F467
:101EE00004C080918B038F3071F410928B03926049
:101EF000977F9093B8011092BB0180E090E060E082
:101F000070E00E94C00C08958823E9F082E060E848
:101F100071E00E94280E83E068E871E00E94280EBC
:101F200084E060E971E00E94280E85E068E971E0D4
:101F30000E94280E86E060EA71E00E94280E87E089
:101F400068EA71E01CC082E060E471E00E94280E43
:101F500083E060E571E00E94280E84E060E671E0B5
:101F60000E94280E85E068E671E00E94280E86E057
:101F700060E771E00E94280E87E068E771E00E9448
:101F8000280E0895882321F082E068EC71E003C0F8
:101F900082E060EC71E00E94280E0895882321F011
:101FA00081E068EB71E003C081E060EB71E00E94CA
:101FB000280E08958093CB010E94FA050895209180
:101FC000B80121FD0EC02B7F21602093B8019093B2
:101FD0009F0180939E017093A7016093A6010E94C8
:101FE000FA050895E0919C01F0919D018E179F07DD
:101FF00011F0EF2BF1F49B0140E050E0A9013327F1
:1020000022278091A2019091A301A091A401B091F7
:10201000A501A070B070282B392B4A2B5B2B209385
:10202000A2013093A3014093A4015093A5010E9403
:10203000FA050895FC0180919C0190919D01E8179B
:10204000F90701F56093BA0160E070E08091A201A8
:102050009091A301A091A401B091A501807090700E
:10206000482B592B6A2B7B2B222311F0616001C076
:102070006E7F4093A2015093A3016093A4017093DB
:10208000A5010DC080919E0190919F01E817F9076D
:1020900041F46093BA015093A7014093A6010E94B6
:1020A000FA0508951F93182F80E06CE00E947B0DC5
:1020B000112309F100D000D00F92EDB7FEB7319691
:1020C00082E0ADB7BEB711968C938DE692E0928315
:1020D00081838091BB0190E08F779070948383839C
:1020E0000E94D20E0F900F900F900F900F9080E0F3
:1020F0000E94380D05C082E068E672E00E942C0F55
:102100001F910895EF92FF920F931F93182F80FF56
:1021100002C083E001C085EA0E94380DE12E11FF64
:1021200002C084E001C085EA0E94380DE2FE02C0D0
:1021300085E001C085EA0E94380DE3FE02C086E01A
:1021400001C085EA0E94380DE4FE02C087E001C0AC
:1021500085EA0E94380D1F910F91FF90EF9008952E
:102160006091A8017091A9018091AA019091AB01A1
:10217000611571058105910561F00E94560988235A
:1021800041F01092A8011092A9011092AA01109298
:10219000AB016091AC017091AD018091AE01909165
:1021A000AF01611571058105910571F00E94560915
:1021B000882351F01092AC011092AD011092AE0143
:1021C0001092AF010E94FA056091B0017091B101C7
:1021D0008091B2019091B30161157105810591055E
:1021E00061F00E945609882341F01092B0011092CC
:1021F000B1011092B2011092B30108958091B8011B
:1022000080FD25C06091A8017091A9018091AA016B
:102210009091AB01611571058105910521F00E9436
:1022200056098823A1F010929F0110929E011092EE
:10223000BE011092BD0110929D0110929C0110925E
:10224000B8011092BF010E94FA0581E0089580E074
:1022500008951F93FC01009769F41092B801109241
:10226000A8011092A9011092AA011092AB010E943C
:10227000FE1048C07091B80171FD44C06093BA016E
:10228000CA01A0E0B0E02091A2013091A3014091E9
:10229000A4015091A50120703070822B932BA42BA8
:1022A000B52B8093A2019093A301A093A401B093B6
:1022B000A5018091590390915A03A0915B03B091BD
:1022C0005C0388519C4FAF4FBF4F81608093A80142
:1022D0009093A901A093AA01B093AB0172FF09C02A
:1022E00071607B7F7093B801F0939F01E0939E0132
:1022F00007C07E7F7093B801F0939D01E0939C012D
:102300000E94FA051F910895DF92EF92FF920F93BA
:102310001F931091CB01112399F081E060E00E949E
:102320007B0D812F81500E941625BC0182E00E9406
:102330002C0F1092CB0188EE93E00E94FF0902C09F
:10234000882319F00E946F0D04C080E060E00E94B5
:102350007B0D80919C0190919D01892BF9F00E9449
:102360006125FC0140919C0150919D0182819381E6
:102370008417950749F4218532858091BD0190919C
:10238000BE012817390751F0538342838091BD0164
:102390009091BE01928781870E944C2620919C01DA
:1023A00030919D0121153105B9F41092A2011092CE
:1023B000A3011092A4011092A5011092A7011092FE
:1023C000A6011092BA011092BB018091B8018F7ED4
:1023D0008093B8011092B9018091B80182FD0DC0BF
:1023E0008091B4019091B501A091B601B091B7016F
:1023F0000097A105B10531F430C082E06BEB72E0CB
:102400000E942C0F8DB79EB707970FB6F8949EBF0A
:102410000FBE8DBFEDB7FEB7319682E0ADB7BEB748
:1024200011968C9388EA92E0928381838091B40123
:102430009091B501A091B601B091B70183839483C7
:10244000A583B6830E94D20EEDB7FEB737960FB6BE
:10245000F894FEBF0FBEEDBF51C02115310531F418
:1024600082E061EA72E00E942C0F21C000D000D00F
:102470000F92EDB7FEB7319682E0ADB7BEB71196B9
:102480008C938CE992E092838183348323830E942E
:10249000D20E8091B8010F900F900F900F900F9077
:1024A00080FF02C081E001C080E20E94380D1091DF
:1024B000B9010E94F705682F863008F0615063303B
:1024C00091F480919C0190919D01892B61F0612F85
:1024D00070E06370707043E0660F771F4A95E1F714
:1024E000605F7D4F08C070E033E0660F771F3A955C
:1024F000E1F7605D7D4F82E00E942C0F80E06CE090
:102500000E947B0D8091B80183FF12C000D000D0E3
:102510000F92EDB7FEB7319682E0ADB7BEB7119618
:102520008C9388E992E0928381838091BB0111C0F2
:1025300000D000D00F92EDB7FEB7319682E0ADB774
:10254000BEB711968C9384E992E092838183809147
:10255000BA0190E08F779070948383830E94D20EAB
:102560000F900F900F900F900F9080919C01909181
:102570009D01892B89F08091B9018370813081F4AC
:1025800087E10E94AB0B882339F080E00E94380D70
:1025900080E060EE71E012C080E20E94380D10C051
:1025A00080E00E94380D8091BA0187FF04C080E06E
:1025B00068E171E003C080E060E271E00E94280EF3
:1025C0000E94F705813049F489E00E943225AC0170
:1025D00081E060E00E94D80D8CC18091B80183FD3C
:1025E00006C080E060E040E050E00E94840D8091F1
:1025F000B80187FD03C000E010E014C080919E0187
:1026000090919F01892B19F001E010E00BC080919F
:10261000B9010E94480F20E030E0853010F021E041
:1026200030E08901F02E81E060E00E947B0D809116
:10263000B4019091B501A091B601B091B701009796
:10264000A105B10509F4B2C08DE00E94AB0B88234F
:1026500029F48EE00E94AB0B882391F100D00F92F9
:1026600082E0EDB7FEB7818388E892E093838283AE
:102670000E94D20E0F900F900F908DE00E94AB0B36
:10268000882369F081E068EB71E00E94280E82E007
:1026900060EC71E00E94280E8EEC9FE00CC081E09F
:1026A00060EB71E00E94280E82E068EC71E00E940D
:1026B000280E82EC9FE06CE271E00E94C00C19C110
:1026C00087E00E943225BC0182E00E942C0F87E047
:1026D0000E9432250E94FC31182F04C080E20E9423
:1026E000380D1F5F1031D0F38091B9010E94480F5F
:1026F00090E0A0E0B0E02091B4013091B5014091AC
:10270000B6015091B70182179307A407B5070CF4DF
:1027100095C081E06BE00E947B0D6091B4017091E7
:10272000B50181E090E0A0E0B0E0062E04C0880F83
:10273000991FAA1FBB1F0A94D2F72091A2013091C2
:10274000A3014091A4015091A50182239323A423C6
:10275000B5230097A105B10519F425EA30E002C0C0
:1027600023E030E08DB79EB707970FB6F8949EBF71
:102770000FBE8DBFEDB7FEB7319682E0ADB7BEB7E5
:1027800011968C938FE792E092838183CB016383D0
:102790009483368325830E94D20EEDB7FEB7379619
:1027A0000FB6F894FEBF0FBEEDBF48C020919E014A
:1027B00030919F012115310539F100D000D00F92E1
:1027C000EDB7FEB7319682E0ADB7BEB711968C93E8
:1027D0008AE792E092838183348323830E94D20E1E
:1027E0000F900F900F900F900F908091A6018F7116
:1027F0000E948210002321F08CE30E94380D2DC02E
:1028000080E20E94380D1CC000D000D00F92EDB7BE
:10281000FEB7319682E0ADB7BEB711968C9381E7D3
:1028200092E0928381838FEB91E0948383830E9473
:10283000D20E0F900F900F900F900F90FF2069F421
:102840008091AC019091AD01A091AE01B091AF012A
:102850000097A105B10509F444C080919E019091B3
:102860009F01892BF1F58091B9010E94480F8530B5
:10287000C0F181E060E00E947B0D86E40E94380D8B
:1028800022E0E22EF12C012D112DDD24D394809134
:10289000A2019091A301A091A401B091A5018E2164
:1028A0009F21A023B1230097A105B10549F0B9E00C
:1028B000BD1518F08D2D805D04C08D2D885001C090
:1028C00085EA0E94380DD394E0E1DE1629F0EE0C83
:1028D000FF1C001F111FDBCF80E20E94380D81E03A
:1028E00006C08091A2018F710E94821080E00E9438
:1028F000840F1F910F91FF90EF90DF900895CF9379
:10290000DF93EB018093B901E82FF0E0EF70F070F6
:10291000E254FD4FE491E093BC016115710559F05B
:10292000CB0160E070E04FEB51E00E94412DD0936D
:10293000BE01C093BD010E94FA05DF91CF910895B9
:10294000AC018091B8018C7F8093B8011092BE01D8
:102950001092BD01662309F043C01092BF0120917F
:102960009C0130919D012115310521F03093A10189
:102970002093A0011092A2011092A3011092A40131
:102980001092A5011092A7011092A60110929F012A
:1029900010929E0110929D0110929C011092B9011B
:1029A00010928B034115510551F18FEFBA010E942E
:1029B00021268091B80181FD22C01092A2011092BF
:1029C000A3011092A4011092A50110929F011092F0
:1029D0009E0110929D0110929C011092B9010DC0B0
:1029E00010928B0360919C0170919D018FEF0E946A
:1029F000E8258091B80181FD02C090E001C091E01E
:102A00008091B8018B7F82608093B801892F0895EF
:102A1000EF92FF920F931F93DF93CF9300D000D0DC
:102A200000D0CDB7DEB77C01FE01319686E0DF0134
:102A30001D928A95E9F7F701208D318D428D538DD6
:102A400062817381211531054105510509F45DC08D
:102A50006115710559F180819181A0E0B0E0821784
:102A60009307A407B50741F0CB01A0E0B0E08217BF
:102A70009307A407B507D1F4D7015C968C915C97B6
:102A80008E7F5C968C935C976D917C918E010F5F2D
:102A90001F4FC8010E94CA2680E065E0A8010E947D
:102AA0003227F7011382128211821082D7018D9191
:102AB0009C91A0E0B0E0F701208D318D428D538DC7
:102AC00082179307A407B50769F4848D91E08927DD
:102AD0008B7F848FD70158961D921D921D921C9258
:102AE0005B9721C081E060E00E947B0D80E00E9446
:102AF0003225BC0182E00E942C0FF701648D6470C6
:102B0000808D918D0E94A01409C0672B39F4D701E4
:102B10005C968C915C9784605C968C93F701108E28
:102B2000118E128E138E26960FB6F894DEBF0FBE4E
:102B3000CDBFCF91DF911F910F91FF90EF9008953E
:102B4000CF92DF92EF92FF920F931F93DF93CF9379
:102B5000CDB7DEB72C970FB6F894DEBF0FBECDBF52
:102B60009C01FE01319686E0DF011D928A95E9F70E
:102B70002531310509F421C326313105ECF42B3020
:102B8000310509F4AAC32C3031056CF42A30310523
:102B90000CF0ACC3213031050CF069C321153105AF
:102BA00009F419C3B9C32F3031050CF053C22D30CD
:102BB00031050CF0EEC137C12332310509F4A5C34C
:102BC0002432310574F42731310509F4F5C0273179
:102BD00031050CF4AEC2C9014997029708F09CC3B5
:102BE00015C02F3831056CF42D3831050CF0D1C1EA
:102BF0002A38310509F476C32C38310509F08CC325
:102C0000C0C12739310509F087C384C38091B80159
:102C100083FF03C01091BB0102C01091BA0100E014
:102C20002931310509F401E0E090BC010E946125E1
:102C3000FC01F7800E946125FC01808184FF35C082
:102C400017FD05C080E0002309F481E0082F002370
:102C500011F001E02CC0812F90E08F779070892BCC
:102C600079F48091B0019091B101A091B201B0913D
:102C7000B3010097A105B10519F4212F205892C086
:102C80008091590390915A03A0915B03B0915C032A
:102C9000845D9E4FAF4FBF4F8093B0019093B101C1
:102CA000A093B201B093B30117C00023A9F00E9412
:102CB000F705833009F075C0812F90E08F77907011
:102CC0002E2D30E0821793070CF06BC0FEE7EF1655
:102CD00071F5FF2071F42BC0812F90E08F779070F9
:102CE000892B09F45EC08EE7E81649F5FF2039F11B
:102CF00000E0A1E0FA1619F460E820E00EC0B2E0AE
:102D0000FB1619F46EE324E108C0E3E0FE1619F4A3
:102D100066E12AE002C060E820E8812F90E030E020
:102D2000002341F08F779070821793075CF4212F76
:102D30002F5F38C08F779070281739071CF0212F2C
:102D4000215030C0462F50E0812F90E08F77907057
:102D5000481759071CF0212F2E7F04C0212F261B56
:102D60002C7F260F211719F00023E1F002C0002369
:102D700061F0822F90E08F7790708417950714F49C
:102D800082E001C084E0280F0DC0822F90E08F7791
:102D900090704817590714F082E001C084E0281BA6
:102DA00001C0212F8091B80183FF03C02093BB0194
:102DB00020782093BA01AEC29091B80197FF1FC04E
:102DC00088E089278093B80183FF0CC08091BA0105
:102DD0008093BB0180788093BA0182E590E160E93D
:102DE00071E00AC08091BB018093BA011092BB01CF
:102DF00080E090E060E070E00E94C00C8BC28091A7
:102E0000B9018370813029F480E060EE71E00E94A6
:102E1000280E8091BA01805880788093BA01809101
:102E2000B801877F6FC2C0909E01D0909F01C114EE
:102E3000D10409F076C0E090B401F090B5010091A2
:102E4000B6011091B7011E141F04100611060CF0F4
:102E500068C08091B9010E94480F90E0A0E0B0E006
:102E60008E159F05A007B1070CF45BC081E090E0D0
:102E7000A0E0B0E00E2C04C0880F991FAA1FBB1F52
:102E80000A94D2F72091A2013091A3014091A401AC
:102E90005091A50182279327A427B5278093A201EB
:102EA0009093A301A093A401B093A5018091B801D0
:102EB00080688093B801F0E1EF16F1040105110577
:102EC0000CF46EC160919C0170919D018E010F5FA9
:102ED0001F4FC8010E94CA262091A2013091A30170
:102EE0004091A4015091A501CA01AA27BB278F7761
:102EF0008B83E7E15695479537952795EA95D1F766
:102F0000822F8F778C8377E0569547953795279555
:102F10007A95D1F72D8380E06DE0A8010E943227D9
:102F20003FC16091B80167FF10C0CD2871F080915A
:102F3000A6019091A70121E030E08227932790938A
:102F4000A7018093A601606119C08091A2019091B0
:102F5000A301A091A401B091A50121E030E040E0DF
:102F600050E082279327A427B5278093A20190934E
:102F7000A301A093A401B093A5016F7E6093B80153
:102F8000C9C180919E0190919F01892B09F0C2C116
:102F9000A9C186E0FE013796DF011D928A95E9F707
:102FA0008091B4019091B501A091B601B091B701A3
:102FB0000097A105B10509F44BC08C0101501040E8
:102FC000000F111FC9018F7790700E9709F40160EF
:102FD00027FF23C01A868091B80183FD05C080E0D9
:102FE00090E060E070E004C082E590E160E971E0AB
:102FF0000E94C00C81E068E371E00E94280E82E02C
:1030000060E471E00E94280E1092B4011092B501A4
:103010001092B6011092B70102C081E08A87802F1A
:103020008F778F83C801880F892F881F990B9195FF
:103030008F778887812F829586958695837089877B
:1030400080E066E0AE01495F5F4F0E94322762C1B7
:1030500027FD60C1022F0D501091B80117FF0AC063
:1030600080919E0190919F01892B21F4213131059E
:103070000CF40C5F8091B9010E94480F081708F00A
:1030800049C10430A0F08091590390915A03A09156
:103090005B03B0915C038C509E4FAF4FBF4F80934A
:1030A000AC019093AD01A093AE01B093AF0117FFB7
:1030B0001DC080919E0190919F01892BB9F082E003
:1030C00090E0A0E0B0E004C0880F991FAA1FBB1FCA
:1030D0000A95D2F72091A6013091A7012827392718
:1030E0003093A7012093A601106120C082E090E0F8
:1030F000A0E0B0E004C0880F991FAA1FBB1F0A956B
:10310000D2F72091A2013091A3014091A4015091E6
:10311000A50182279327A427B5278093A201909326
:10312000A301A093A401B093A5011F7E1093B80141
:10313000F1C08091B4019091B501A091B601B09118
:10314000B7010097A105B105A1F18091B80182FDF9
:1031500030C00E94F705833019F58091BC01282FFB
:1031600030E040E050E08091B4019091B501A09131
:10317000B601B091B701281739074A075B0744F435
:103180002093B4013093B5014093B6015093B70139
:103190008091BA0180789091B401892B8093BA0113
:1031A0001092B4011092B5011092B6011092B701BD
:1031B000B1C080E060E243E00BC08091B80187FFBE
:1031C00004C080E060E242E003C080E060E240E0F2
:1031D0000E9448279FC08091B80187FF12C080914C
:1031E000A0019091A101009709F496C0A0E0B0E081
:1031F0008093B4019093B501A093B601B093B70149
:103200001EC082FF21C08091B4019091B501A091B0
:10321000B601B091B7010097A105B105A9F486E008
:103220000E94E0248091B4019091B501A091B60173
:10323000B091B7010097A105B10509F46DC08CE903
:1032400091E00E94081568C08091B4019091B50189
:10325000A091B601B091B7010097A105B10539F46D
:103260008FEF0E94E02481E00E94841155C0790113
:103270000027F7FC0095102F6091B4017091B50103
:103280008091B6019091B7012AE030E040E050E033
:103290000E94BD31E60EF71E081F191FB0E0EB16A5
:1032A000B8E2FB06B0E00B07B0E01B0724F080910A
:1032B000B80186FF31C0E0E0EE16E0E4FE06E0E093
:1032C0000E07E0E01E0744F5E092B401F092B5016C
:1032D0000093B6011093B7011DC08CE991E00E94E4
:1032E000081518C08091B8018F770CC01092B401F6
:1032F0001092B5011092B6011092B7018091B801F9
:103300008B7F80688093B80105C08091BA01807876
:103310008093BA010E94FA052C960FB6F894DEBF8E
:103320000FBECDBFCF91DF911F910F91FF90EF9016
:10333000DF90CF900895FB0157FD02C021E004C04B
:10334000509541955F4F20E08330910541F18430E5
:10335000910534F48130910501F1029751F523C0B4
:103360008430910519F0059721F50AC081818F5F9E
:10337000818390E084179507E4F0222351F00DC07B
:1033800081818150818390E08417950794F02223F6
:1033900021F0842F815081830CC011820AC01282D7
:1033A0001382168A06C090E08281882309F491E096
:1033B000928380E090E008958230910519F00397A0
:1033C00051F403C02FEF3FEF08C083E090E040E0EE
:1033D00050E00E949B1920E030E0C90108951F933E
:1033E000182F0E94550FFC01848D112311F0806469
:1033F00001C08F7B848F1F910895CF93DF93EB01E2
:1034000082309105B1F18330910534F40097B1F029
:10341000019709F048C005C0863091050CF043C003
:1034200023C00E946125FC01808190E024E09695F4
:1034300087952A95E1F78170898335C081E060E046
:103440000E947B0D8981825F0E94322500D00F92FD
:1034500022E0EDB7FEB72183938382830E94D20ED0
:103460000F900F900F901FC042E050E00E949B19F8
:103470001AC08A81882389F08981882331F00E94CB
:103480006125FC018081806105C00E946125FC01ED
:1034900080818F7E80830E944C2690E08A818823E1
:1034A00009F491E09A8380E090E0DF91CF91089554
:1034B000CF93DF93EB018230910581F18330910549
:1034C0002CF4009781F00197C9F504C0863091056E
:1034D000ACF51FC00E946125FC018781898384307F
:1034E00068F119822BC081E060E00E947B0D898128
:1034F000865F0E94322500D00F9222E0EDB7FEB722
:103500002183938382830E94D20E0F900F900F909D
:1035100015C044E050E00E949B1910C08A818823A6
:1035200039F00E9461252981FC0127830E944C26E5
:1035300090E08A81882309F491E09A8380E090E00A
:10354000DF91CF9108950F931F93CF93DF938C0159
:103550000E94580FEC01009731F482E062ED72E0B6
:103560000E942C0F18C000D000D00F92EDB7FEB70C
:10357000319682E0ADB7BEB711968C938EEC92E097
:1035800092838183D483C3830E94D20E0F900F90C5
:103590000F900F900F900115110521F082E0B801F6
:1035A0000E942C0FCE01DF91CF911F910F910895B2
:1035B0000F931F93CF93DF938C010E94550FEC0163
:1035C0000115110521F002301105D9F518C080E070
:1035D00090E00E94A31A892BA1F181E060E00E9493
:1035E0007B0D89A19AA1892B11F081E001C082E0B5
:1035F0000E943225BC0182E00E942C0F22C08A81E9
:103600009B81892BF1F488819981892BD1F089A143
:103610009AA1892BB1F081E060E00E947B0D83E0EC
:103620000E943225BC0182E00E942C0F84EF91E0C1
:103630000E94FF0989A19AA10E94F72B1AA219A240
:103640001BA280E090E0DF91CF911F910F91089530
:103650000F931F93CF93DF93EB018230910509F411
:10366000A1C0833091053CF4009709F43EC0019756
:1036700009F0D4C00CC08430910509F444C08430F2
:1036800091050CF488C0059709F0C8C061C00E947C
:10369000550FFC0180819181892B09F4BFC09F01E6
:1036A0002D5D3F4FAE014B5E5F4FDE011A9660E22B
:1036B00017C0F9018081882359F0E8EDF2E0949178
:1036C000981721F031969923D1F702C08C9301C04D
:1036D0006C93F9018081882311F02F5F3F4F119681
:1036E000A417B50730F31C9299C080E090E00E94C7
:1036F000A31A81E060E00E947B0D2A9682E0BE0161
:103700000E94C10E8BC08981A82FB0E0FB01EA0F97
:10371000FB1F228548ED52E0FA0180E09491921758
:1037200031F03196992311F08F5FF8CF8FEF8F5FD3
:10373000E82FFF27E7FDF095E852FD4F849188239D
:1037400011F4FA018491AC0FBD1F1A968C9366C0D8
:103750008981A82FB0E0FB01EA0FFB1F2285E8ED6D
:10376000F2E080E09491921729F03196992339F094
:103770008F5FF8CF882319F0E82FE15001C0EFE206
:10378000FF27E7FDF095E852FD4FE491AC0FBD1F18
:103790001A96EC9343C083E090E04AE050E00E9428
:1037A0009B193CC00E94550F8C01FC0182819381C2
:1037B000892BA1F58A81882349F489E08B8381E0F4
:1037C000888F19821F8A8A838E8B28C089818F5F98
:1037D00089838F8B8B3010F11B821A821E8A98018D
:1037E0002D5D3F4FD901FE013A968CE001900D927C
:1037F0008150E1F7F80181A192A160817181009768
:1038000021F0458D0E94802C06C0CB01F801658D0A
:10381000A9010E94372DF80192A381A380E090E0D6
:10382000DF91CF911F910F9108954F925F926F9208
:103830007F928F929F92AF92BF92CF92DF92EF9240
:10384000FF920F931F93DF93CF9300D000D000D04F
:10385000CDB7DEB78C016B010E94550F7C010230A1
:10386000110509F48BC00330110544F4011511054D
:1038700039F10130110509F027C105C006301105E5
:103880000CF022C135C0DC015D962C915D97922F22
:1038900093705C968C9186FF04C0992329F494E080
:1038A00003C0992309F491E02695269523702350AF
:1038B00083E0989FC0011124280FF601218304C1E1
:1038C00081E060E00E947B0D8DE693E00E94A31AE8
:1038D000892B09F4F9C0D60111966C918AE0689F92
:1038E000B0011124675F7C4F82E00E942C0FECC076
:1038F000FC01848D86FD03C049E050E002C04AE02F
:1039000050E0C801B6010E949B19D7018D919C918E
:103910008F3F9105D9F0D0F0F6018181882311F411
:1039200086E08183D7015C968C9186FD06C0F60106
:103930008181863010F488E08183D60111968C91C4
:103940001197863018F489E011968C93F7018081E5
:1039500091818050984208F4B7C0D60111968C919D
:103960001197882319F489E011968C93F6018181CF
:10397000893008F0A9C089E08183A6C0DC011296D5
:103980008D919C911397892B09F09EC0F60182813D
:10399000882309F490C08D909C9011978114910414
:1039A00009F492C05D968C910E943E0F5C01D60195
:1039B00011964C91842F63E00E94DC31292F30E076
:1039C000220F331F220F331F842F0E94DC31182F48
:1039D0001F5F122B143009F410E0F70141A052A030
:1039E000812F0E943E0FD7015E964C91242F30E02C
:1039F0002F773070FC01E29FC001E39F900DF29F92
:103A0000900D1124B5010E94E8314078462BD70172
:103A10005E964C935AE0A52EB12CAC0CBD1C43E233
:103A2000642E712C6E0C7F1CC501B3010E940C32F8
:103A3000FE01319686E0DF011D928A95E9F7882D17
:103A40008F778983C401880F892F881F990B9195DF
:103A50008F778A831F771B838FEF64E0AF010E940B
:103A6000322781E060E00E947B0D80E00E943225D9
:103A7000BC0182E00E942C0F80E090E060E040E01A
:103A800050E00E9429118FEFB4010E9421264114B9
:103A9000510469F0F70160817181C201458D950182
:103AA0000E94802CD70192969C938E939197C3018C
:103AB000B5010E940C3290E0F6018281882309F45E
:103AC00091E0D60112969C9380E090E026960FB686
:103AD000F894DEBF0FBECDBFCF91DF911F910F9144
:103AE000FF90EF90DF90CF90BF90AF909F908F901E
:103AF0007F906F905F904F900895AF92BF92CF925A
:103B0000DF92EF92FF920F931F93DF93CF93CDB786
:103B1000DEB727970FB6F894DEBF0FBECDBF7B018F
:103B20008230910509F46CC08330910534F400971C
:103B3000F1F0019709F009C10CC08430910509F436
:103B400049C0843091050CF454C0059709F0FDC0BC
:103B500047C09B01265F3F4FC90160E270E04BE028
:103B600050E00E940532D70155961C92EEC0FB0131
:103B70008281882309F4E9C08181882309F4E5C0A2
:103B80008B01065F1F4F90E060E070E0A8010E948B
:103B9000412D00D000D00F92EDB7FEB7319622E054
:103BA000ADB7BEB711962C9320E733E03283218363
:103BB000948383830E94D20E0F900F900F900F90EA
:103BC0000F9081E060E00E947B0D82E0B8010E94CE
:103BD000C10EBBC0FB01818190E00E947C2C05C01E
:103BE000FB01818190E00E94782CD70111968C9383
:103BF000ACC083E090E040E050E00E949B19A5C07B
:103C000090E0FB018281882309F491E0D7011296AC
:103C10009C930E94550F8C01F7018281882371F0DB
:103C2000D80191968D919C919297009729F480E00C
:103C300090E00E947C2CF701818387C0BAE0AB2E14
:103C4000B12CAE0CBF1CD70111968C9190E0BE0137
:103C50006F5F7F4FA5010E94412D6C01F801848D9B
:103C600082FF08C0C601A0E0B0E0808F918FA28FD4
:103C7000B38F68C0D8018D919C911197009721F066
:103C800015969C938E931497F801138612861382CF
:103C90001282D80116961D921D921D921C921997A0
:103CA00011961C921E925C968C915C978C7F5C9610
:103CB0008C938FEFB6010E942126F80180819181BB
:103CC000892B81F1FE01329686E0DF011D928A95F3
:103CD000E9F78C2D8F778A83C601880F892F881F7B
:103CE000990B91958F778B8389818F778C838FEF59
:103CF00064E0AF010E94322781E060E00E947B0D0A
:103D000080E00E943225BC0182E00E942C0F80E0FE
:103D100090E060E040E050E00E9429118FEFB60192
:103D20000E942126F80180819181892B59F0C801D8
:103D30008396B5010E940C32D70111968C91F8013F
:103D400081A312A22FEF3FEF02C020E030E0C901B3
:103D500027960FB6F894DEBF0FBECDBFCF91DF918F
:103D60001F910F91FF90EF90DF90CF90BF90AF9099
:103D700008950F931F93CF93DF93EC018B0100976E
:103D800031F097FD40C002970297E8F536C081E018
:103D900060E00E947B0DD80112968C91882359F423
:103DA00082E066E873E00E942C0F82E060E873E036
:103DB0000E942C0F22C00E946B25EDB7FEB73797EB
:103DC0000FB6F894FEBF0FBEEDBF319622E0ADB73F
:103DD000BEB711962C9324E733E0328321836383AB
:103DE0007483858396830E94D20EEDB7FEB7379613
:103DF0000FB6F894FEBF0FBEEDBFCE01B80140E094
:103E000050E00E949B1980E090E0DF91CF911F91DC
:103E10000F910895CF93DF93EB018230910509F460
:103E20004AC08330910534F4009799F0019709F066
:103E300056C005C0863091050CF051C037C00E94B5
:103E40006125DC0114968C9163E00E94DC3189834A
:103E500046C081E060E00E947B0D998183E0989FDD
:103E6000802D11240E94F80C82E090E00E94FF094E
:103E700081B763E00E94DC31898300D000D00F92CB
:103E8000EDB7FEB7319692E0ADB7BEB711969C93F1
:103E90002FE833E032832183838314820E94D20E81
:103EA0000F900F900F900F900F9019C04FEE5FEF93
:103EB0000E949B1914C08A81882359F00E946125B1
:103EC000298143E0249F90011124FC0124830E9456
:103ED0004C2690E08A81882309F491E09A8380E05F
:103EE00090E0DF91CF9108950F931F93CF93DF93CD
:103EF000FC018B01EA0180819181892B21F0858D64
:103F00008370833081F081E060E00E947B0D85E06A
:103F10000E943225BC0182E00E942C0F80E0033019
:103F2000110519F521C00E94F7058330E9F00E94C0
:103F3000F7058230C9F00630110531F480E060E207
:103F400043E00E9448270EC081E060E00E947B0DA4
:103F500086E00E943225BC0182E00E942C0F1A826A
:103F60001B821E8A80E001C081E0DF91CF911F910A
:103F70000F910895CF92DF92EF92FF920F931F93CC
:103F8000DF93CF9300D000D000D0CDB7DEB77C0157
:103F90008B010E94550F6C01B701A8010E94741F8C
:103FA000882309F4F5C042E0E416F10409F4B3C033
:103FB00083E0E816F1044CF4E114F104A9F1A1E066
:103FC000EA16F10409F0E4C010C0B4E0EB16F10405
:103FD00009F46CC0E4E0EE16F1040CF494C0F5E0D2
:103FE000EF16F10409F0D4C077C08EEF9FEFD8012F
:103FF0005A969C938E9359972091D5013091D60172
:10400000C90101978050944020F4F801358324833E
:1040100005C0D8011596FC92EE92149780E094E0CA
:10402000F80197838683B4C0D80112968C918823B7
:1040300009F4AEC081E060E00E947B0DF8012481AC
:10404000358137FF14C000D00F9282E0ADB7BEB704
:1040500011968C93119787E993E013969C938E9316
:1040600012970E94D20E0F900F900F9018C000D0A0
:1040700000D00F92EDB7FEB7319682E0ADB7BEB774
:1040800011968C9383E993E0928381833483238315
:104090000E94D20E0F900F900F900F900F9083E020
:1040A000F801878B81E0808F868B72C0D8011496CF
:1040B0008D919C911597019615969C938E931497CC
:1040C00016962D913C91179782179307C4F0159679
:1040D0003C932E93149713C0D80114968D919C9104
:1040E0001597019715969C938E9314971816190699
:1040F00034F081E090E015969C938E93149781E0C4
:10410000F801838345C083E090E0B80140E050E0CF
:104110000E949B193DC091E0D80113969C93139780
:1041200012968C911297882381F114962D913C91CF
:1041300015971216130664F53093D6012093D50116
:10414000F60180818F77898380819181880F892F03
:10415000881F990B91958F778A8314968C91815043
:104160008F778B8321503040220F232F221F330B58
:10417000822F87708C831D821E828FEF68E0AE01D4
:104180004F5F5F4F0E94322703C0D80112969C9365
:1041900080E090E026960FB6F894DEBF0FBECDBF4C
:1041A000CF91DF911F910F91FF90EF90DF90CF9013
:1041B0000895CF92DF92EF92FF920F931F93DF93B8
:1041C000CF9300D000D000D0CDB7DEB78C017B01FB
:1041D0000E94550F6C01B801A7010E94741F88232B
:1041E00009F43DC10230110509F4CAC003301105BC
:1041F00044F40115110561F10130110509F02FC1D9
:104200000DC00430110509F4B9C0043011050CF4D7
:104210001FC10530110509F022C115C18EEF9FEFB6
:10422000D7015A969C938E9359972091D50130913E
:10423000D601C90101978050944020F4F7013583DD
:1042400024830DC1D70115961C930E93149707C1B3
:10425000F7018281882309F402C181E060E00E94B5
:104260007B0DD70112968C91882309F4F8C081E068
:1042700060E00E947B0D00D000D00F92EDB7FEB73A
:10428000319612E0ADB7BEB711961C9384EB93E064
:1042900092838183D70114968D919C911597948375
:1042A00083830E94D20E0F900F900F900F900F906B
:1042B000F7018381843099F400D00F92ADB7BEB777
:1042C00011961C93119780EB93E013969C938E9319
:1042D00012970E94D20E0F900F900F901AC000D02C
:1042E00000D00F92EDB7FEB73196ADB7BEB71196BD
:1042F0001C938CEA93E092838183D70118968C916A
:10430000838314820E94D20E0F900F900F900F9013
:104310000F90F701818D928D97FD04C082E064EAD1
:1043200073E00CC08E5F9F4F21F482E06CE973E074
:1043300005C084E00E943225BC0182E00E942C0F5F
:1043400081E0D70158968C93589756968C93569740
:1043500013968C91813078F0833020F08450823035
:1043600050F404C083E0F701878B79C088E0D7015F
:1043700057968C9374C0F701168A71C084E064C0AC
:10438000F7018281448155818823A1F481E08383F0
:1043900080E094E097838683415054403CF081E074
:1043A00090E0D70115969C938E93149781E0F701C6
:1043B000828355C05093D6014093D50141155105D4
:1043C000F1F1D70113968C91139781508230B8F197
:1043D000F60180818F77898380819181880F892F71
:1043E000881F990B91958F778A8314968C911497D7
:1043F00081508F778B8318963C91832F90E0807843
:1044000090709595879541505040440F452F441F1B
:10441000550B242F2770282B2C833F773D831E823A
:104420008FEF67E0AE014F5F5F4F0E943227D701E9
:1044300013961C920E94770D2FEF3FEF12C081E080
:10444000F70183830CC081E0D70113968C9307C0DA
:1044500083E090E0B70140E050E00E949B1920E02B
:1044600030E0C90126960FB6F894DEBF0FBECDBF6F
:10447000CF91DF911F910F91FF90EF90DF90CF9040
:104480000895CF92DF92EF92FF920F931F93CF93F5
:10449000DF937C01162F0E946F0D0E9461256C0135
:1044A0001E3008F069C0C12FD0E08E01000F111F2F
:1044B000000F111F0C0F1D1F0E5F1E4FD70112960C
:1044C0008C91882311F080E001C081E00E94380DBA
:1044D000F6018581823069F0833099F0BE01E4E015
:1044E000660F771FEA95E1F78130A9F466547C4F97
:1044F00014C054E0CC0FDD1F5A95E1F7C657DB4FCF
:1045000007C044E0CC0FDD1F4A95E1F7C65ADA4FE9
:1045100082E0BE0103C0665D794F82E00E942C0FED
:10452000D70112968C91882389F4F801848187FD44
:104530000DC081E060E00E947B0DD80114968C9143
:104540000E943225BC0182E00E942C0FD8011296F5
:10455000ED91FC911397309721F080E090E0B70146
:104560000995F7018689882329F0808D67890E9443
:10457000220E02C00E94770DDF91CF911F910F9103
:10458000FF90EF90DF90CF9008952F923F924F923F
:104590005F926F927F928F929F92AF92BF92CF92D3
:1045A000DF92EF92FF920F931F93DF93CF93CDB7DC
:1045B000DEB76B970FB6F894DEBF0FBECDBFD82E17
:1045C0008CE08D1508F4E1C1DE0111968BE1FD014F
:1045D00011928A95E9F7A8958D2D90E0FC01EE0FD8
:1045E000FF1FEE0FFF1FE80FF91FEE5FFE4F028067
:1045F000F381E02D309721F081E090E0BD01099535
:104600008E010F5F1F4FC8016D2D0E9441220E9435
:10461000550F55E0A52EB02EC12E4AE0242E3EEFB8
:10462000432E3FEF532E22E0322E9FEF892E9FE73D
:10463000992E8BE0682E712C6C0E7D1EDA9C700119
:10464000112487010E5F1E4F0E94FE050E94CF0BB2
:10465000AC018531910509F474C1863191057CF472
:104660008A30910509F4F9C08B30910524F499231F
:104670000CF006C1E9CF8B30910531F78AC0893142
:10468000910591F08A31910544F48631910509F440
:1046900061C187319105C1F67CC08A319105B9F1BC
:1046A0008232910589F66BC18B81882369F0D8012C
:1046B0001296ED91FC911397309719F084E090E0F9
:1046C0003CC18A818F5F32C01F8AF701EE5FFE4FC7
:1046D0009081D394BCE0BD1524F08581891709F43D
:1046E00046C0E2E0F1E060E0292F332727FD309556
:1046F000808190E08217930711F4D62E38C06F5F47
:104700006D3011F03596F4CFDD24DA9430C08B8112
:10471000882371F0D8011296ED91FC911397309790
:1047200019F085E090E009C18A8181508A8327C110
:104730001F8AF701EE5FFE4F9081DA94D7FC04C028
:1047400035978081891799F0EEE3F1E00CE0D02EE7
:10475000292F332727FD3095808190E0821793071A
:1047600031F0DA94BFEFDB1611F03597F5CF8D2DD0
:1047700090E0FC01EE0FFF1FEE0FFF1FE80FF91F87
:10478000EE5FFE4F0280F381E02D309709F05BC0B1
:10479000F6C0F80191819923E9F1A92FB0E0FD015C
:1047A000E353FE4F80811816BCF0E2E0F1E020E018
:1047B000492F552747FD5095808190E08417950734
:1047C00011F4822F06C02F5F2D3011F03596F4CFF3
:1047D0008FEFA353BE4F8C93D8011196EC91F0E06C
:1047E000E353FE4F80810E94C522282F332727FDE7
:1047F0003095F8018181E82FF0E0E353FE4FC901C5
:1048000037FF04C088279927821B930B808337FFCB
:10481000B6C00EC0D8011296ED91FC911397309757
:10482000A9F082E090E06B2D7C2D099597FF02C0E6
:10483000D194ACC08B81882309F0A1C0D801129615
:10484000ED91FC91139781E090E077C090E08B812F
:10485000882309F491E09B8392C08B81882309F41B
:1048600095C0D8011296ED91FC911397309731F0D5
:1048700083E090E06B2D7C2D0995DCCF1B827FC0FF
:104880008C818430D1F1853040F48230E9F083307E
:1048900060F4813009F073C008C0883031F089308D
:1048A000E1F1853009F06BC02AC08F819885892B92
:1048B00011F498868F828F819885841795070CF460
:1048C0005EC01E821D823C828D819E819C01B3E070
:1048D000220F331FBA95E1F7880F991F280F391F50
:1048E000240F351F37FD4BC08F81988582179307A2
:1048F0000CF445C03E832D8342C01986AC82898565
:10490000829DC0011124840F951F8F3F910509F0EE
:1049100008F489875B8E4A8E32C08A81F301E80FE2
:10492000F11D842F805D8083D8011296ED91FC915A
:104930001397309721F182E090E06B2D7C2D099543
:104940001EC080E00E94CB0680E060E240E00E9452
:10495000482715C0D8011296ED91FC911397309716
:1049600029F086E090E06B2D7C2D0995F80180817F
:10497000882329F483E290E00E94A01507C08B2DC4
:104980009C2D6D2D0E94412259CEDD248D2D6B96DC
:104990000FB6F894DEBF0FBECDBFCF91DF911F9150
:1049A0000F91FF90EF90DF90CF90BF90AF909F90CE
:1049B0008F907F906F905F904F903F902F900895D1
:1049C0001F93182F0E947925803871F180E068EEDE
:1049D00071E00E94280E81E060EE71E00E94280ED6
:1049E0008091CD018D3010F01092CD0117FD04C0E3
:1049F000812F0E94C5220EC08091CD010E94C52248
:104A0000992787FD909597FF03C0909581959F4FBB
:104A10008093CD0180E068E171E00E94280E81E082
:104A200068E371E00E94280E1F910895882319F011
:104A30002EE337E015C00E946125FC01858182309C
:104A400039F0833041F0813049F42AEF36E008C074
:104A50002BE037E005C02CE137E002C02DE237E063
:104A6000C90108951F93182F803118F02EE83BE0FC
:104A700025C00E946125FC018581823059F0833078
:104A800081F08130A9F481E1189F90011124225B0B
:104A9000384F14C081E1189F90011124225A374FDA
:104AA0000DC081E1189F900111242259364F06C094
:104AB00081E1189F900111242258354FC9011F919F
:104AC000089587ED91E008959091D701982309F01A
:104AD00091E0892F08952CEF3FEF41E050E04BBF6C
:104AE000F90127913791479156915070B901CA0148
:104AF00008958FEF9FEFA1E0B0E0ABBFFC0187917D
:104B0000823029F4079902C080E8089582E0089570
:104B1000FC01848D81FD02C020E006C020E0808180
:104B20009181892B09F021E0822F0895FC01848D69
:104B300081FD02C020E006C020E082819381892BA4
:104B400009F021E0822F0895F89488E181BD8BE07F
:104B500081BDFFCFBF92CF92DF92EF92FF920F9372
:104B60001F93CF93DF93082F6B01EA014115510585
:104B700029F10E94550F7C0110E086E0B82E80E0FC
:104B8000602FA6010E943227B0928C0302C00E94BF
:104B9000FE05C701FE010995882321F480918C034D
:104BA0008823A9F70E94D626811110E0C701FE01D3
:104BB0000995882319F41F5F1A3008F3DF91CF910C
:104BC0001F910F91FF90EF90DF90CF90BF900895CD
:104BD000DF93CF9300D000D000D0CDB7DEB7611502
:104BE000710531F14115510519F1FE01319686E04B
:104BF000DF011D928A95E9F7862F8F778983660FEB
:104C0000672F661F770B7195862F8F778A83842F86
:104C10008F778B83440F452F441F550B5195842F5D
:104C20008F778C8382E0BF0146E955E20E94AA2576
:104C300026960FB6F894DEBF0FBECDBFCF91DF91A1
:104C40000895DF93CF9300D000D000D0CDB7DEB76A
:104C500061157105C1F0FE01319686E0DF011D92FC
:104C60008A95E9F7862F8F778983660F672F661FEE
:104C7000770B7195862F8F778A8381E0BF0148E893
:104C800055E20E94AA2526960FB6F894DEBF0FBE05
:104C9000CDBFCF91DF910895CF93DF93C0E0D0E0F7
:104CA000CE010E947B34FE01E952FE4F60818617DF
:104CB00019F0CE010E948334A8952196C032D10507
:104CC00079F7DF91CF91089580959091D70198233E
:104CD0009093D7010E944C2608959091D701982B6C
:104CE0009093D7010E944C2608958093DC010E9486
:104CF0004C2608959091DC01973008F091E080E116
:104D0000E7EDF1E0DF011D928A95E9F788E18093F4
:104D1000DB019093DC010E944C26089587ED91E021
:104D200060E070E040E250E00E946B348091D90175
:104D30009091DA018F5F9F4F11F40E947A26809143
:104D4000DC01873010F01092DC018AEF9FEFA1E0C8
:104D5000B0E0ABBFFC019791892F81508E3F10F4DA
:104D600090936F000895FC0120E090E037E081917E
:104D7000982780E097FF03C0990F932701C0990FF0
:104D80008F5F8830B9F72F5F283089F797FD9095AE
:104D9000892F0895FC01862F8F778083660F672FF8
:104DA000661F770B71956F77618308958091FC0181
:104DB000882319F01092FC0181E0089520914401AC
:104DC000309145019093450180934401C9010895B4
:104DD0009093FA018093F90181E08093FB0108959B
:104DE000E091F701F091F801309709F009950895E5
:104DF0008091430108950F931F93DF93CF93CDB715
:104E0000DEB729970FB6F894DEBF0FBECDBFDA012B
:104E100080914301806889836A83FE0133969E01F5
:104E2000275F3F4F109721F08D918F77808301C0CE
:104E300010823196E217F307A9F78E010F5F1F4F1B
:104E4000C8010E94B3268987C8010E946908299673
:104E50000FB6F894DEBF0FBECDBFCF91DF911F918B
:104E60000F9108950F931F93CF93DF93082F162F61
:104E7000EA0102C00E94FE05802F612FAE010E9450
:104E8000FB268823B9F3DF91CF911F910F910895ED
:104E9000DF93CF9300D000D000D0CDB7DEB7FE01B6
:104EA000319696E0DF011D929A95E9F74983AF01AB
:104EB0000E94322726960FB6F894DEBF0FBECDBFF4
:104EC000CF91DF910895FF920F931F93CF93DF93BC
:104ED000082FEB014115510519F42FEF3FEF47C0A3
:104EE00080914401909145015093450140934401C4
:104EF0009093F8018093F7011092FB018EEF9FEFE2
:104F00009093FA018093F90110E094E0F92E0023C8
:104F100029F080E0602FAE010E943227F0928C03CE
:104F200002C00E94FE059091FB01992321F480911B
:104F30008C038823B1F78091FC01882319F010922B
:104F4000FC0110E0992319F41F5F183000F38091E1
:104F5000F7019091F80190934501809344011092DC
:104F6000F8011092F7012091F9013091FA01C9017D
:104F7000DF91CF911F910F91FF900895DF92EF92F3
:104F8000FF920F931F93DF93CF93CDB7DEB729978F
:104F90000FB6F894DEBF0FBECDBF8E010F5F1F4F5F
:104FA00024E0E22E29E2F22EDD24D3941CC0C801B5
:104FB0000E94B32699858917B1F41BC0D092FC01D9
:104FC00012C08091440190914501892B21F4F09207
:104FD0004501E0924401E0914401F0914501309790
:104FE00011F0C8010995C8010E949308892BF9F6B0
:104FF00004C08A81863029F7E1CF29960FB6F8944C
:10500000DEBF0FBECDBFCF91DF911F910F91FF90FB
:10501000EF90DF9008952F923F924F925F926F92A0
:105020007F928F929F92AF92BF92CF92DF92EF9238
:10503000FF920F931F93DF93CF93CDB7DEB72997DE
:105040000FB6F894DEBF0FBECDBF0E946B259B014B
:10505000AC0110E8612E1FE3712E812C912C62228D
:10506000732284229522B7E095948794779467946D
:10507000BA95D1F7A12CA0ECBA2EAFE1CA2ED12C53
:10508000A222B322C422D522FEE0D594C794B794BD
:10509000A794FA95D1F7E12CF12CE0EE0E2F112D0B
:1050A000E222F3220423152375E115950795F79461
:1050B000E7947A95D1F76FE7262E312C412C512CAD
:1050C00022223322442255222DC0A8958A81843081
:1050D00049F5CE0101960E94B3269985891711F5ED
:1050E00041C08D8190E0A0E0B0E0681679068A06A4
:1050F0009B06C1F48C8190E0A0E0B0E0A816B90650
:10510000CA06DB0679F48B8190E0A0E0B0E0E816F7
:10511000F9060A071B0731F489818F7780934301D1
:1051200081E007C0CE0101960E949308892B69F6A1
:1051300080E029960FB6F894DEBF0FBECDBFCF91A9
:10514000DF911F910F91FF90EF90DF90CF90BF9074
:10515000AF909F908F907F906F905F904F903F9017
:105160002F9008958E8190E0A0E0B0E028163906D7
:105170004A065B06B9F6B5CF0F931F93DF93CF9323
:10518000CDB7DEB729970FB6F894DEBF0FBECDBFFF
:10519000209143012068298323E02A83282F2F7739
:1051A0002B83880F892F881F990B91958F778C837C
:1051B000862F8F778D83852F869586958E8367FFC3
:1051C00002C080648E83CA0103E0969587950A9594
:1051D000E1F78F778F83842F8295807788878E0180
:1051E0000F5F1F4FC8010E94B3268987C8010E9424
:1051F000890829960FB6F894DEBF0FBECDBFCF91B8
:10520000DF911F910F910895AF92BF92CF92DF92DD
:10521000EF92FF920F931F93DF93CF9300D000D0B4
:1052200000D0CDB7DEB76C010E94550F5C01D601EE
:1052300011966C91862F90E0FC013397E132F105D5
:1052400008F08EC2EA5BFF4FEE0FFF1F0590F4914E
:10525000E02D0994F60182810E94CB06D6011796B3
:105260008C9184700E94EF197BC2F501008111813D
:10527000D60113968C91139790E09695982F8827D6
:105280009795879512962C9130E0822B932B0817D7
:10529000190709F065C20E94FE10C8010E94A22FE2
:1052A0005FC2F6018381E82FF0E0F695FE2FEE272E
:1052B000F795E795D60112968C91129790E0E82B1E
:1052C000F92B15968C911597382F330F330F20E05B
:1052D00016968C911697482F50E04F77507013E038
:1052E000440F551F1A95E1F717968C9190E080773F
:1052F000907074E0959587957A95E1F7482B592B36
:10530000422B532B683041F4CF01BA010E94DF0FCA
:1053100080918B0382602FC080918B03816080938A
:105320008B03D60117968C9180FD05C080918B036D
:10533000826080938B03D60114966C911497159616
:105340008C9186FD6068CF010E9429110E94660F32
:1053500007C2F601668170E07695762F662777950D
:105360006795858190E0682B792B84810E947F145A
:1053700080918B03846080938B03E8CFD6011496D1
:105380004C91149750E015966C91159770E07695B6
:10539000762F66277795679516962C911697922FFC
:1053A0009295990F990F907C80E0682B792B13963A
:1053B0008C91139790E09695982F882797958795CD
:1053C00012962C9130E0642B752B822B932B0E942C
:1053D000F20F80918B038860CECFF601628113813A
:1053E0008581E82FF0E0D60116964C911697179616
:1053F0008C911797282F30E014960C91E6FD0068E9
:10540000FE2FEE27FF0FFF0F50E04F77507083E025
:10541000440F551F8A95E1F7C90180779070B4E079
:1054200095958795BA95E1F7482B592B812F90E0F8
:105430009695982F88279795879570E04E2B5F2B30
:10544000E3E036952795EA95E1F72170862B972BB7
:10545000602F0E941A1084C1F50121A132A12115EB
:10546000310569F0822F8F778983220F232F221F26
:10547000330B3195822F8F778A8318E00EC0D501C8
:105480008C918F7789838D919C91880F892F881FAC
:10549000990B91958F778A8310E0F501848D80FDBB
:1054A00010610E946B25262F2F772B83A7E09695FE
:1054B000879577956795AA95D1F7262F2F772C8317
:1054C000F7E09695879577956795FA95D1F7262F0A
:1054D0002F772D83E7E09695879577956795EA95E1
:1054E000D1F76770612B6E838FEF6BE0AE014F5F7A
:1054F0005F4F0E94322734C10E946B257B018C01D3
:105500009B01AC012F77307040705070D60114961B
:105510008C9190E0A0E0B0E0281739074A075B07BC
:1055200009F054C1A801970120783F734070507072
:1055300067E056954795379527956A95D1F7F60117
:10554000858190E0A0E0B0E0281739074A075B07A3
:1055500009F03CC1A80197012070307C4F71507058
:105560009EE056954795379527959A95D1F7868170
:1055700090E0A0E0B0E0281739074A075B0709F080
:1055800025C1278180E090E0A0EEB0E0E822F9227A
:105590000A231B2385E116950795F794E7948A95CE
:1055A000D1F7822F90E0A0E0B0E087709070A070FB
:1055B000B070E816F9060A071B0709F007C18381D6
:1055C000682F70E07695762F6627779567958281AC
:1055D00090E0682B792B6115710509F4F7C02695C9
:1055E00026952695122F20FF0BC0A5014D5D5F4F1C
:1055F000CB0160E070E00E94412DBC01009721F0DA
:10560000809143010E942126D5018D919C91119793
:10561000892B09F4DBC011FFD9C05C968C915C9793
:1056200081605C968C93D2C0F601838190E0969560
:10563000982F882797958795228130E0822B932B8E
:1056400090938E0380938D038BC0D60113968C911B
:10565000139790E09695982F88279795879512969F
:105660002C91129730E0822B932B9093910380938F
:10567000900314968C91149780939E0315968C91A9
:1056800015978093920316968C9180939303809143
:105690008F03816012C022E030E0F601E20FF31FB9
:1056A0008081F901EE56FC4F80832F5F3F4F2730FA
:1056B000310599F780918F03826080938F0350C0EA
:1056C000F601828180939903838180939A03848178
:1056D00080939B03858180939C0380918F038460DA
:1056E000ECCFD60115968C9115978823C9F11396A6
:1056F0008C911397482F50E05695542F4427579577
:10570000479514962C911497922F9295990F990F73
:10571000907C80E0482B592B12968C9190E0482B7E
:10572000592B40FD02C067E601C062E7CA019695A9
:1057300087950E94DD2F14C00E94A425F601828166
:105740000E94DA0F0DC0D60112968C91882329F0A1
:105750000E946125FC01848101C080E00E94F80C58
:10576000D6012C9130E02F7730708091430190E08A
:105770002817390749F480918C03882329F08091F8
:105780008C03815080938C03F501848D81FD06C0CC
:1057900080E090E060E040E050E016C084FF0EC082
:1057A000D50112968D919C911397009739F01A9616
:1057B0004D915C911B975E966C9106C0F5014681F8
:1057C000578180819181668D0E94BC2826960FB6F4
:1057D000F894DEBF0FBECDBFCF91DF911F910F9127
:1057E000FF90EF90DF90CF90BF90AF900895DF9340
:1057F000CF9300D000D000D0CDB7DEB7FE013196F8
:1058000026E0DF011D922A95E9F7282F2F772983BB
:10581000880F892F881F990B91958F778A838FEF37
:1058200063E1AF010E94322726960FB6F894DEBFDF
:105830000FBECDBFCF91DF910895DF92EF92FF921F
:105840000F931F93DF93CF9300D000D000D0CDB73C
:10585000DEB7E62EFE01319626E0DF011D922A9585
:10586000E9F7282F2F772983880F892F881F990B15
:1058700091958F778A838FEF9FEF90938E0380931C
:105880008D0310E0FE2E0F2F35E0D32E16C08FEFC4
:105890006E2D4F2D502F0E943227D0928C0302C0C4
:1058A0000E94FE0580918D0390918E0397FF04C0A6
:1058B00080918C038823A1F71F5F80918D039091C5
:1058C0008E0397FF02C01A3011F720918D0330919B
:1058D0008E03C90126960FB6F894DEBF0FBECDBF6A
:1058E000CF91DF911F910F91FF90EF90DF9008957E
:1058F00062E10E941D2C089561E10E941D2C089513
:105900008F929F92AF92BF92CF92DF92EF92FF92CF
:105910000F931F93DF93CF9300D000D000D0CDB76B
:10592000DEB7FC0179016115710509F48AC0211502
:10593000310509F486C06E010894C11CD11C86E0B3
:10594000D6011D928A95E9F7CB01880F892F881F10
:10595000990B9195BFE79B2E982214E1AFE7AA2EF1
:10596000A6227FE7B72EB42265E0862E8E2F8F7792
:105970008983EE0FEF2FEE1FFF0BF1958E2F8F77A0
:105980008A83163171F0173128F4143171F0153112
:1059900031F505C0173139F0183109F50AC090E02A
:1059A0000CC080E008C080E005C0AB829C82BD8254
:1059B00016C083E08D5F982F9D5FF701E90FF11D01
:1059C00080818B83892F8F5FF701E80FF11D908114
:1059D0009C838F5FF701E80FF11D80818D8310920A
:1059E0008E0310928D0300E015C08FEF612FA6018A
:1059F0000E94322780928C0302C00E94FE05809193
:105A00008D0390918E03892B21F480918C03882340
:105A1000A1F70F5F80918D0390918E03892B11F474
:105A20000A3019F780918D0390918E03892B49F0EC
:105A3000E0918D03F0918E031F5F193109F096CF2D
:105A400002C0E0E0F0E0CF0126960FB6F894DEBF8A
:105A50000FBECDBFCF91DF911F910F91FF90EF90BF
:105A6000DF90CF90BF90AF909F908F900895FC01F2
:105A7000A62F9A0180E090E0BF014A2F0E94802C5F
:105A80000895AF92BF92CF92DF92EF92FF920F9361
:105A90001F93DF93CF9300D000D000D0CDB7DEB7F7
:105AA0009C018B017A0101978F5F934008F06CC0D5
:105AB000FE01319686E0DF011D928A95E9F7822F7B
:105AC0008F778983220F232F221F330B3195822F4B
:105AD0008F778A8310928F03DD24BE2ECF2E8FE026
:105AE000A82E1EC08FEF60E14B2D5C2D0E94322747
:105AF000A0928C0302C00E94FE0580918F03873024
:105B000021F080918C038823B1F780918F03873037
:105B100031F082B790E08C599F4F0E94FF09D394D7
:105B200080918F03873019F0BAE0DB16D9F68091A7
:105B30008F03873021F4809192038F3759F4011538
:105B4000110511F0F8011082E114F104E9F0D70118
:105B50001C921AC00115110521F080919E03F801D5
:105B60008083E114F10459F0D701E2E9F3E08BE01E
:105B700001900D928150E1F7D7011B961C92209164
:105B800090033091910302C020E030E0C9012696D5
:105B90000FB6F894DEBF0FBECDBFCF91DF911F913E
:105BA0000F91FF90EF90DF90CF90BF90AF9008954E
:105BB000982F1092A0038091A00380939F0380915F
:105BC0009F038093C2038091C2038093C103119A03
:105BD0001098199A189882E08BB9983008F091E0E3
:105BE000E92FF0E0EE0FFF1FE556F44FA591B491B9
:105BF000653010F465E003C0693008F068E04F7D5F
:105C00006550660F453411F4606203C04F3409F4E7
:105C10006063223008F068608B2F992787FD9A9582
:105C20008F7080939000A9B96093950088EB8AB932
:105C300080E090E008951F920F920FB60F920BB67E
:105C40000F9211248F939F93EF93FF939091C10331
:105C50008091C203981711F4559812C0E091C203C5
:105C6000F0E0E156FC4F84A18CB98091C2038F5FB4
:105C70008093C2038091C203883010F01092C20357
:105C8000FF91EF919F918F910F900BBE0F900FBEE0
:105C90000F901F9018951F920F920FB60F920BB690
:105CA0000F9211242F933F938F939F93EF93FF9322
:105CB00020919F038091A00330E090E00197281786
:105CC000390741F080919F038F3179F48091A003CF
:105CD000882359F48091A0038F5F8093A003809163
:105CE000A003803210F01092A003E0919F03F0E037
:105CF0008CB1E156FC4F828380919F038F5F80932C
:105D00009F0380919F03803210F010929F03FF91B8
:105D1000EF919F918F913F912F910F900BBE0F901C
:105D20000FBE0F901F90189527E0813D9207C0F19C
:105D30002FE0813A920710F481E01EC023E28932FD
:105D4000920710F482E018C026E3813B920710F41A
:105D500083E012C026E48135920710F484E00CC081
:105D600028E8893B920710F485E006C0895D964DCE
:105D700010F087E001C086E0789420E030E05E9982
:105D800002C020E030E02F5F3F4FA89597E220311E
:105D90003907A8F368E04EE421E00E94D82D089569
:105DA00080E0EACF8330C9F0843028F4813061F09C
:105DB000823080F40CC08530B1F0853088F08630B8
:105DC000A9F08730C9F415C020E639E017C020EBF0
:105DD00034E014C020EC32E111C020E835E20EC0FE
:105DE00020E438E30BC020E03BE408C020E036E9C3
:105DF00005C020E031EE02C020E030E0C901089586
:105E000039B120919000922F80E0232F30E0282B91
:105E1000392B4BE95BE060E0FA01859194918217A0
:105E2000930729F06F5F4E5F5F4F6830A9F7862FA9
:105E30000E94D22E0895482FA89503C0559A7894B1
:105E4000A8952091C1038091C20330E090E00197B2
:105E50002817390799F38091C103873021F4809185
:105E6000C203882359F3E091C103F0E0E156FC4FEF
:105E700044A39FB7F8948091C1038F5F8093C103BF
:105E80008091C103883010F01092C1039FBF559AD2
:105E900080E090E0089590919F038091A00398176F
:105EA00019F42FEF3FEF15C0E091A003F0E0E156A9
:105EB000FC4F9281F8948091A0038F5F8093A003A0
:105EC0008091A003803210F01092A003292F30E0BF
:105ED0007894C9010895CF92DF92EF92FF920F93C9
:105EE0001F93CF93DF93E82E162F042FF52E6AEC25
:105EF0000E94590E8E2D612F0E94590E802F9F2DCA
:105F0000EC0185E0C82ED12CCC0EDD1E0FC018810F
:105F1000812F8A5C843028F48E2D6BEC0E94590E00
:105F20001F708E2D612F0E94590E2196CC15DD0514
:105F300071F7DF91CF911F910F91FF90EF90DF905C
:105F4000CF900895DF93CF9300D000D000D0CDB78D
:105F5000DEB7FE01319626E0DF011D922A95E9F7B2
:105F600099838A8380E063E0AF010E946B2F2696BD
:105F70000FB6F894DEBF0FBECDBFCF91DF9108956D
:105F8000DF93CF9300D000D000D0CDB7DEB7FE01B5
:105F9000319696E0DF011D929A95E9F7898380E0BA
:105FA00062E0AF010E946B2F26960FB6F894DEBF19
:105FB0000FBECDBFCF91DF910895DF93CF9300D077
:105FC00000D000D0CDB7DEB7FE01319626E0DF016C
:105FD0001D922A95E9F799838A836F776B8380E016
:105FE00066E0AF010E946B2F26960FB6F894DEBFD5
:105FF0000FBECDBFCF91DF910895EF92FF920F9327
:106000001F93DF93CF93CDB7DEB762970FB6F894A7
:10601000DEBF0FBECDBF162F882309F094C180913B
:1060200007028823B1F06091FD017091FE0180911B
:10603000FF01909100026C5E7F4F8F4F9F4F0E9437
:106040005609882331F0109207021092080210922C
:1060500009028091590390915A03A0915B03B0917A
:106060005C038093FD019093FE01A093FF01B09328
:1060700000021A3C41F4109207021092080281E0DB
:106080008093090260C180910902882309F45BC1F1
:106090001B3C21F481E08093080255C180910802E5
:1060A0008111106C1092080280910702E82FF0E035
:1060B000E350FE4F14838F5F80930702863008F40D
:1060C00042C10E94550F8C0190910102933009F456
:1060D000B4C0943030F4913059F1923008F055C08A
:1060E0000AC0953009F4C5C0953008F4B4C09630A4
:1060F00009F01FC1E8C080E06CEC0E94590ED80185
:1061000016968D919C9117979C012E7F3F7736951F
:10611000279580FD3068F801868D8F833887298721
:106120000E94F7058A871C861B8680E060E027C0F6
:1061300080E06CEC0E94590ED80111968C91119759
:106140008F835C915D964C915D97242F30E0237096
:10615000307093968C91992787FD9095282B392B39
:10616000232B11F480E001C080E858878987842FB1
:106170000E943E0F8A871C861B8680E061E0AE018C
:10618000495F5F4F0E946B2FD8C09091020280E060
:1061900020910302BC01620F711D9091050280E005
:1061A00020910602820F911DAC01440F551F4E7FB6
:1061B0005F7797FD41606115710519F4F801608101
:1061C0007181F0E460307F0708F0B3C0D8018D9191
:1061D0009C916817790739F4CB016091040220E0A3
:1061E0000E941A106DC0862F8F778983660F672FE4
:1061F000661F770B7195862F8F778A8390910402A3
:10620000892F8F778B83852F869586958C8397FF33
:1062100002C080648C83CA0133E0969587953A95D5
:10622000E1F78F778D83842F829580778E8380E04E
:1062300063E0AE014F5F5F4F41C09091020280E08A
:1062400020910302820F911D60E00E94A014882318
:1062500009F46FC035C040910202442329F0842F15
:106260008250823008F065C080E060E20E944827DA
:1062700027C03091020220E080910302280F311DD7
:10628000FE01319686E0DF011D928A95E9F7822FA3
:106290008F778983C901880F892F881F990B919562
:1062A0008F778A83832F82958695869583708B83DB
:1062B000809104028C8380E066E0AF010E94322767
:1062C00080E06CEC38C03091020220E08091030243
:1062D000280F311D8E01035F1F4FF80111929A950F
:1062E000E9F7F22EE32EC801B9010E94CA2689E11E
:1062F000B80140EB51E30E9463278C018235910580
:1063000069F08335910524F48734910591F406C032
:106310008736910519F08237910559F480E06CECCD
:106320000E94590E602F6F778F2D9E2D0E94DD2FBA
:1063300004C080E06DEC0E94590E1092070210928A
:1063400008021092090262960FB6F894DEBF0FBEE3
:10635000CDBFCF91DF911F910F91FF90EF900895E6
:10636000FC018181893121F0CF010E94F02608953E
:10637000848190E00E94E8260895629FD001739F77
:10638000F001829FE00DF11D649FE00DF11D929FD1
:10639000F00D839FF00D749FF00D659FF00D992710
:1063A000729FB00DE11DF91F639FB00DE11DF91F34
:1063B000BD01CF0111240895991B79E004C0991FF4
:1063C000961708F0961B881F7A95C9F7809508954F
:1063D000AA1BBB1B51E107C0AA1FBB1FA617B7070B
:1063E00010F0A61BB70B881F991F5A95A9F7809527
:1063F0009095BC01CD010895FC0105900020E9F7BE
:10640000809590958E0F9F1F0895DC0101C06D93BC
:1064100041505040E0F70895FB01DC0101900D92DE
:106420000020E1F708950F931F93DF93CF93CDB72B
:10643000DEB72E970FB6F894DEBF0FBECDBF8C012E
:1064400086E08C831A8309838FEF9FE79E838D8379
:10645000CE0101960E946532EF81F885E00FF11FB1
:1064600010822E960FB6F894DEBF0FBECDBFCF912F
:10647000DF911F910F9108950F931F93DF93CF9397
:10648000CDB7DEB72E970FB6F894DEBF0FBECDBFE7
:106490008C018EE08C831A8309838FEF9FE79E83A4
:1064A0008D83CE0101960E946532EF81F885E00F61
:1064B000F11F10822E960FB6F894DEBF0FBECDBF2F
:1064C000CF91DF911F910F9108952F923F924F929C
:1064D0005F926F927F928F929F92AF92BF92CF9274
:1064E000DF92EF92FF920F931F93DF93CF93CDB77D
:1064F000DEB72B970FB6F894DEBF0FBECDBF3C01C1
:106500002B015A01FC0117821682838181FD03C091
:106510006FEF7FEFC6C19AE0892E1E010894211CFF
:10652000311CF3012381F20123FD859123FF819129
:106530002F01882309F4B2C1853239F423FD8591F6
:1065400023FF81912F01853229F490E0B3010E944D
:10655000A634E7CF982FFF24EE249924FFE1FF15FE
:10656000D0F09B3269F09C3228F4903259F093328B
:1065700091F40EC09D3249F0903369F441E024C09B
:1065800052E0F52A84E0F82A28C098E0F92A25C0CC
:10659000E0E1FE2A22C0F7FC29C0892F80538A300F
:1065A00070F4F6FE05C0989C902C1124980E15C02E
:1065B000E89CE02C1124E80EF0E2FF2A0EC09E3287
:1065C00029F4F6FC6BC140E4F42A07C09C3619F4A8
:1065D00050E8F52A02C0983649F4F20123FD95915E
:1065E00023FF91912F01992309F0B8CF892F85546A
:1065F000833018F08052833038F444E050E0A40E29
:10660000B51E5FE359830FC0933631F0933779F0AD
:10661000933509F056C020C0F5018081898342E09E
:1066200050E0A40EB51E610101E010E012C0F501BA
:10663000C080D180F6FC03C06FEF7FEF02C0692DF0
:1066400070E042E050E0A40EB51EC6010E949B34EB
:106650008C015FE7F52214C0F501C080D180F6FC03
:1066600003C06FEF7FEF02C0692D70E042E050E0A1
:10667000A40EB51EC6010E9490348C0150E8F52A84
:10668000F3FE07C01AC080E290E0B3010E94A63476
:10669000EA948E2D90E008171907A8F30EC0F601B2
:1066A000F7FC8591F7FE81916F0190E0B3010E94A4
:1066B000A634E110EA94015010400115110579F754
:1066C000EAC0943611F0993669F5F7FE08C0F50175
:1066D000208131814281538184E090E00AC0F5013C
:1066E000808191819C01442737FD4095542F82E0A1
:1066F00090E0A80EB91E9FE6F92257FF09C05095F9
:106700004095309521953F4F4F4F5F4FE0E8FE2A6F
:10671000CA01B901A1012AE030E00E94D234D82E8A
:10672000D21840C0953729F41F2D1F7E2AE030E093
:106730001DC01F2D197F9F3661F0903720F49835CA
:1067400009F0ACC00FC0903739F0983709F0A6C0F7
:1067500004C028E030E00AC0106114FD146020E19C
:1067600030E004C014FD166020E132E017FF08C0DD
:10677000F501608171818281938144E050E008C01D
:10678000F50180819181BC0180E090E042E050E021
:10679000A40EB51EA1010E94D234D82ED2188FE7C4
:1067A000F82EF122F6FE0BC05EEFF522D91438F474
:1067B000F4FE07C0F2FC05C08FEEF82202C01D2DCA
:1067C00001C0192DF4FE0DC0FE01ED0DF11D8081FB
:1067D000803319F499EEF92208C01F5FF2FE05C05C
:1067E00003C08F2D867809F01F5F0F2DF3FC14C0B6
:1067F000F0FE0FC01E1510F09D2C0BC09D2C9E0CA2
:10680000911A1E2D06C080E290E0B3010E94A634CA
:106810001F5F1E15C0F304C01E1510F4E11A01C05D
:10682000EE2404FF0FC080E390E0B3010E94A63481
:1068300002FF1DC001FD03C088E790E00EC088E59F
:1068400090E00BC0802F867891F001FF02C08BE2B0
:1068500001C080E2F7FC8DE290E0B3010E94A63413
:1068600006C080E390E0B3010E94A6349A94D91444
:10687000C0F3DA94F101ED0DF11D808190E0B301D8
:106880000E94A634DD20A9F706C080E290E0B301A3
:106890000E94A634EA94EE20C1F743CEF30166814C
:1068A0007781CB012B960FB6F894DEBF0FBECDBF1C
:1068B000CF91DF911F910F91FF90EF90DF90CF90DC
:1068C000BF90AF909F908F907F906F905F904F9010
:1068D0003F902F900895DC01CB01FC01E199FECFA0
:1068E00006C0FFBBEEBBE09A31960DB20D9241504F
:1068F0005040B8F70895E199FECF9FBB8EBBE09A58
:1069000099278DB30895262FE199FECF9FBB8EBBAB
:106910002DBB0FB6F894E29AE19A0FBE0196089546
:10692000FC010590615070400110D8F7809590955A
:106930008E0F9F1F0895FC0161507040019001105F
:10694000D8F7809590958E0F9F1F08950F931F93F2
:10695000CF93DF938C01EB018B8181FF1BC082FF02
:106960000DC02E813F818C819D812817390764F4E9
:10697000E881F9810193F983E88306C0E885F98508
:10698000802F0995892B31F48E819F8101969F83F9
:106990008E8302C00FEF1FEFC801DF91CF911F91CF
:1069A0000F910895FA01AA27283051F1203181F181
:1069B000E8946F936E7F6E5F7F4F8F4F9F4FAF4F07
:1069C000B1E03ED0B4E03CD0670F781F891F9A1F1A
:1069D000A11D680F791F8A1F911DA11D6A0F711DCE
:1069E000811D911DA11D20D009F468943F912AE0DA
:1069F000269F11243019305D3193DEF6CF010895C2
:106A0000462F4770405D4193B3E00FD0C9F7F6CFF2
:106A1000462F4F70405D4A3318F0495D31FD4052BA
:106A2000419302D0A9F7EACFB4E0A6959795879550
:106A300077956795BA95C9F700976105710508952F
:106A40009B01AC010A2E06945795479537952795DB
:106A5000BA95C9F7620F731F841F951FA01D089573
:046A6000F894FFCFD8
:106A6400FFFF00010000FF0000D920080000BA1F4A
:106A7400FF00020000FF00000A1FFF0000B91EFF14
:106A84000000DC19FF01007D1DFF0100151CFF0142
:106A940000281BFF0100D81AFF0200581AFF020049
:066AA400FD19FFFF0429AB
:00000001FF
